:020000040800F2
:10000000D81D0020010100083D570008C53F000829
:10001000715500081910000829840008000000002C
:100020000000000000000000000000005D68000803
:10003000BB2E000800000000F95C0008856B00087A
:100040001B010008B55A00081B0100081B0100082D
:100050001B0100081B0100081B0100081B01000810
:100060001B0100081B0100081B0100081B01000800
:100070001B0100081B010008E12900081B01000802
:100080001B0100081B01000859070008017F000838
:10009000AD7F00081B010008411000081B0100088B
:1000A000156C0008ED6C00081B0100081B0100081E
:1000B000F16C0008D96F0008357200081B010008B8
:1000C0001B0100081B0100081B0100081B010008A0
:1000D0001B010008517E00081B0100081B010008DD
:1000E0001B0100081B0100081B010008DFF80CD0F1
:1000F00000F0F4FA00480047559A0008D81D002087
:100100000648804706480047FEE7FEE7FEE7FEE7B1
:10011000FEE7FEE7FEE7FEE7FEE7FEE7A16B00086D
:10012000ED0000082DE9F0410024061B254671F181
:10013000000605DA01240027D0EB070067EB010178
:10014000161E73F1000605DA0027D2EB070201251F
:1001500067EB030300F0DEF986460E4617469C4621
:10016000AC4204D00025D0EB050E65EB010624B1AE
:100170000020D2EB000760EB030C704631463A4694
:100180006346BDE8F08140EA01039B0703D009E024
:1001900008C9121F08C0042AFAD203E011F8013B73
:1001A00000F8013B521EF9D2704710B5002200E062
:1001B000521C835C8C5CA34201D1002BF8D1D8B2D5
:1001C000E1B2401A10BD80EA010210B502F000430E
:1001D000400022D04A001FD0010E01EB1261C0F393
:1001E0005600C2F3560240F4000042F40002A0FBA5
:1001F000022000047F39140400D0401C50EA124051
:1002000001D44000491EC2B20C0604EBD010401CC1
:100210004008802A02D003E0002010BD20F0010039
:10022000002900DA0020184310BD2DE9FE4F81EAB5
:10023000030404F0004421F0004100944FF0000B4F
:1002400023F0004350EA01045ED052EA03045BD07D
:10025000C3F30A54C1F30A552C44A4F2F3340194B5
:10026000A0FB0254C1F3130141F48011C3F3130343
:1002700043F4801301FB024400FB034E840A970AF7
:1002800044EA815447EA8357A4FB076802958D0A24
:1002900005FB07854FEA932C04FB0C542705029DB0
:1002A0004FEA065847EA1637B5EB08056EEB070C20
:1002B000870E920E47EA811742EA8312A7FB0201DA
:1002C000B6EB0B0164EB00042B0D43EA0C335E1814
:1002D00044EB1C50DA465146E7FB0201C5F3130418
:1002E0004FEA0B3343EA14534FEA0432019C43EACA
:1002F0000603A4F10C040294009CCDE900B400F0C4
:100300009FF903B0BDE8F08F00200146F9E72DE921
:10031000F04D81EA030404F0004B21F0004514463F
:100320004FF0000A23F0004150EA050220D054EAC1
:1003300001021DD0C5F30A570246C5F31303C1F3EA
:100340001300C1F30A5640F4801543F48013A7EB61
:100350000608101BD64608F2FD3873EB050002D3E1
:1003600008F1010801E092185B41B8F1000F03DACF
:1003700000200146BDE8F08D00204FF480110646B4
:1003800084460EE0171B73EB050705D3121B63EBC6
:10039000050306434CEA010C49084FEA3000921865
:1003A0005B4150EA0107EDD152EA030012D082EA24
:1003B000040083EA0501084305D0101BAB4106D2B7
:1003C0000122002306E000224FF0004302E06FF01C
:1003D000010253101AEB06004CEB085110EB0A0017
:1003E00041EB0B01BDE8F04D00F01BB970B521F0F9
:1003F000004303430CD0C1F30A550024D5EB040598
:1004000064EB0403D617AD1AB34102DB00200146AA
:1004100070BD201841EB025170BDC10F80EAE07041
:100420000844CA079623002100F0CDB89623002285
:10043000114600F0C8B80EB5C10F80EAE07008445C
:10044000CA07002140F233438DE80E000A460B46EE
:1004500000F0F6F803B000BD0EB540F23341029152
:100460000021CDE900110A460B4600F0E9F803B07F
:1004700000BD00F0004220F00040C10DC0F31600A6
:1004800040F400007F2901DA00207047962903DC40
:10049000C1F19601C84001E096398840002AF4D0A5
:1004A0004042704770B5C1F30A5201F00045002484
:1004B000C1F3130140F2FF3341F480119A4201DA93
:1004C000002070BD40F233439A42A2F2334203DC73
:1004D000524200F05FF800E090402C43F1D04042DF
:1004E00070BDC1F30A5210B5C1F3130140F2FF33DE
:1004F00041F480119A4201DA002010BD40F23343EA
:100500009A42A2F2334203DC524200F043F810BD9B
:10051000904010BD2DE9F05F0546002092469B46B5
:1005200088460646814640241BE028464146474609
:10053000224600F02FF853465A46C01A914110D374
:1005400011461846224600F016F82D1A67EB0108EE
:100550004F4622460120002100F00DF817EB00095C
:100560004E41201EA4F10104DFDC484631462A46F4
:100570004346BDE8F09F202A04DB203A00FA02F14E
:10058000002070479140C2F1200320FA03F3194381
:1005900090407047202A04DB203A21FA02F0002123
:1005A000704721FA02F3D040C2F120029140084383
:1005B000194670470029A8BF7047401C490008BF72
:1005C00020F00100704710B4B0FA80FC00FA0CF083
:1005D00050EA010404BF10BC704749B1CCF12004BB
:1005E00021FA04F411FA0CF118BF01212143084348
:1005F000A3EB0C01CB1D4FEA00614FEA102042BF74
:10060000002010BC704700EBC35010440029A4BF69
:1006100010BC7047401C490008BF20F0010010BC0E
:10062000704710B5141E73F1000408DA401C41F144
:10063000000192185B411A4301D120F0010010BD66
:100640002DE9F04D92469B4611B1B1FA81F202E0DC
:10065000B0FA80F220329046FFF78DFF04460F4635
:1006600040EA0A0041EA0B0153465A46084313D0B8
:10067000114653EA010019D0C8F140025046FFF775
:1006800089FF05460E46504659464246FFF773FF1E
:10069000084305D0012004E020463946BDE8F08D2E
:1006A0000020054346EAE0762C4337430A98630569
:1006B000E40AA0EB08000022FD0A44EA47540A308D
:1006C00002D500200146E9E7010510196941DDE97D
:1006D000084500196941BDE8F04DA2E7064C074DF9
:1006E00006E0E06840F0010394E807009847103402
:1006F000AC42F6D3FFF7FEFC40BC000860BC00082B
:1007000070B58C1810F8015B15F0070301D110F8D3
:10071000013B2A1106D110F8012B03E010F8016B00
:1007200001F8016B5B1EF9D12B0705D40023521E83
:100730000DD401F8013BFAE710F8013BCB1A921CEB
:1007400003E013F8015B01F8015B521EF9D5A142E9
:10075000D8D3002070BD00002DE9F0415B4C4FF470
:1007600090652946204600F042FA002871D02946BB
:10077000204600F0C9F856490888401C088001212D
:10078000204600F013FB534842F21072B0F85810A4
:10079000914202D2491CA0F8581009F08FFB4E4D2F
:1007A000B5F91410B5F9120008F02CF84B4CA5F867
:1007B00056002080A16820468847A088A5F85800E8
:1007C00005F026F809F07AFC454E464C30780828AA
:1007D00036D045F6AC30606042F6EF60A06042F281
:1007E000C400E0604048008A2080208E6080A16BB9
:1007F0003C488847208E40F21C7180003B4C00EB47
:1008000081006887207A4FF0000740073DD5384DBA
:1008100040F21A61E888401C80B2E880884232D3F6
:100820004FF48051334803F051F801282BD132495D
:10083000EF8032480A780A2A0ED2438853B10BE07F
:1008400041F2130060604FF48060A06040F61B50DE
:10085000C7E718E0521C0A70D1B2022913D84188A8
:10086000002910D1A16821F00401A1602449CA889F
:1008700022F40062CA80017821F00201017021494E
:1008800049F681600880BDE8F08130780A2818D2E6
:10089000DFE800F0170613050A050D171113F2E73C
:1008A000BDE8F04108F084B90AF0BEFB05E0BDE800
:1008B000F04104F031B908F0A3FEBDE8F04109F0C1
:1008C00055BD01F0E7FD84F8BA70DCE70024014073
:1008D00058070020380100204C000020400700206D
:1008E0004F070020CC000020F0010020A8020020CB
:1008F000D80A0020000C014073020020F2050020FD
:10090000100C0020442C01406FEA11210160704757
:100910000029816802D041F0010101E021F00101CC
:10092000816070470029816802D041F4807101E044
:1009300021F48071816070472DE9F041854E92B0BD
:10094000304600F011F90BA800F03FFA01214FF4F6
:10095000C06005F065FA00248DF831404FF4602046
:10096000CDE90D044FF4A0204FF00A080B900127A9
:100970008DF83C808DF830700BA9304600F086F978
:10098000754D8DF831408DF830708DF83C700BA9A5
:10099000284600F07BF901231A460F21304600F06B
:1009A000C6F9022201231146304600F0C0F90123A6
:1009B00003221946304600F0BAF90123042200212F
:1009C000304600F0B4F9012305220321304600F03F
:1009D000AEF9012306220821304600F0A8F90123D0
:1009E00007220A21304600F0A2F9012308220B2138
:1009F000304600F09CF9012309220D21304600F019
:100A000096F901230A220421304600F090F90121D1
:100A1000304600F084F90121284600F080F90123D6
:100A20001A460521304600F055F901231A460621E1
:100A3000284600F04FF90021304600F0CBF84FF483
:100A4000E041284600F0C6F80121304600F0B8F831
:100A50000121284600F0B4F80121304600F0A6F844
:100A60000121284600F0A2F80121304600F09EF94D
:100A70000121284600F09AF940F61451374806F053
:100A8000B0FE12208DF8400002208DF841008DF854
:100A900042408DF8437010A804F07EFE01224FF40E
:100AA0009061304600F0E8F801213046FFF73AFF48
:100AB00001213046FFF72CFF01212846FFF728FFD0
:100AC000304600F06EF9304600F09FF80028FAD169
:100AD000304600F075F9304600F082F80028FAD16F
:100AE000284600F05EF9284600F08FF80028FAD179
:100AF000284600F065F9284600F072F80028FAD17F
:100B00000121084605F068F9154D284601F0A4FFBB
:100B1000684602F044F80F4801A94C300090114893
:100B200081E811018020CDE904404000069080005A
:100B30000790202008904FF44050CDE90904694601
:100B4000284602F00FF80121284601F079FF12B083
:100B5000BDE8F0810024014000280140002C014044
:100B600008000240B80200200D4910B5884202D1A9
:100B7000012144150AE00B49884202D101210415E4
:100B800004E0094988420AD10121CC03204605F03E
:100B900053F92046BDE81040002105F04DB910BDC5
:100BA0000024014000280140003C014000298168E8
:100BB00002D041F4801101E021F48011816070477E
:100BC0000029816802D041F4004101E021F4004194
:100BD00081607047826822F4E0420A438260704775
:100BE000014600208968490700D50120704710B5EB
:100BF0000246002054680B0AC9B20C401168194221
:100C000002D0002C00D0012010BD014600208968D0
:100C1000090700D50120704738B501211C2005F0D7
:100C2000FFF8EF20ADF8000000248DF80340032505
:100C30008DF8025069460D4802F0CAFD0120ADF85A
:100C400000008DF803408DF802506946084802F014
:100C5000BFFD3B20ADF800008DF803408DF8025039
:100C60006946044802F0B4FD38BD000000080140A8
:100C7000000C014000100140002A4268C9B201D0B6
:100C80000A4300E08A4342607047000010B54268A2
:100C90000E4B0C791A400B6842EA0422134343605E
:100CA00083680B4A1340D1E9024222434C7943EA5C
:100CB00044031A438260C26A097C22F47002491E0E
:100CC000C9B242EA0151C16210BD0000FFFEF0FF4F
:100CD000FDF7F1FF70B5072409290AD9C568A1F10C
:100CE0000A0606EB4606B440A543B3401D43C56063
:100CF00007E0056901EB4106B440A543B3401D433D
:100D00000561836BC3F30154121B921C02EB820436
:100D10001F22A2409343A1400B43836370BD826BAB
:100D2000491E22F4401242EA01518163704770B5B6
:100D3000072409290AD9C568A1F10A0606EB460667
:100D4000B440A543B3401D43C56007E0056901EB0E
:100D50004106B440A543B3401D4305611F23072A44
:100D600009D2446B521E02EB820293409C43914095
:100D70000C43446370BD0D2A09D2046BD21F02EBF1
:100D8000820293409C4391400C43046370BDC46A4B
:100D90000D3A02EB820293409C4391400C43C462A3
:100DA00070BD816841F00801816070470029816849
:100DB00002D041F4A00101E021F4A001816070475C
:100DC000816841F004018160704700210160017178
:100DD00041718160C160012101747047002800DA0F
:100DE0004042B0F5803F02DB4FF6FF70704780B2A3
:100DF0007047000070B51E4C214694F83800B1F8D9
:100E0000425006281ED9B4F84A10B4F84C00A1EBA1
:100E1000000202F10902122A04D8FFF71DFB00228A
:100E2000144B0AE0884204D2FFF716FB0022124B53
:100E300003E0FFF711FB0022104BFFF7F6F9FFF775
:100E400050FB09E005D12846FFF706FB0C4A0D4B85
:100E5000F3E70D4951F82000C5EB45116063B0EB95
:100E6000410F03D9C5EB45104000606370BD000021
:100E70005C04002000003440000033400000354096
:100E80006766666666E64B40B8B2000810B50C4C63
:100E90002078400713D5FFF7ADFF0A49A08E0880E0
:100EA00008483038018821F010010180001F0188B6
:100EB00041F010010180207820F00400207010BD66
:100EC0005C04002040040040F0B4254A254C002179
:100ED000137A02F1380033B1B4F9023041F2CD0592
:100EE000AB4211DC11721E4E83683836C3F3C00763
:100EF000C3F300253668AF4211D1350706D5DD05AD
:100F000006D443F0080305E0A180C162F0BC70473D
:100F100023F008038360518301231372F4E790F8F0
:100F20004A40D4B9104C646CB4F5966F15DC3407A4
:100F300013D4548BB4F5FA6F02D2641C5483E5E7E2
:100F40000A4A65F3C303147824F001041470518035
:100F500011828360F0BC08F04BB95183D6E70000E2
:100F600070020020F205002038010020C00A002095
:100F7000012180F82E104FF4AF6101861F214186B8
:100F800045F271518186704770B506464089204B05
:100F9000204C4FF40051002580B362887AB1012AB9
:100FA0000CD1E188491C89B2E1803289914205D394
:100FB0006580E580FF2801D0401E708170BD70887B
:100FC0002288904201D9012200E00022184602F056
:100FD00088FC7088B18801442088401C80B2208041
:100FE0008142EBD82580A088401C80B2A080F18887
:100FF0008842E3D301206080A58070BDFFE7002216
:10100000184602F06EFCA580E58025806580F4E737
:1010100000100140D8050020FEE7000010B5074C85
:101020000021204600F06AF80121204600F066F811
:101030002046BDE81040022100F060B80064004086
:1010400010B50D4C0B49204600F06AF809492046BE
:10105000891C00F065F80949204600F061F8084C49
:10106000206807F0C5FD002106A008F025FE2060DD
:1010700010BD00000200F010006400407000F0306D
:101080005C0800206465765F63616E3100000000DB
:1010900070B51848017861F30704417861F30F24B3
:1010A000817861F31744C17861F31F640179407955
:1010B00061F3070560F30F2502F092F90E4E3046FA
:1010C00002F00CF9A1B2304602F044F9210CB01C38
:1010D00002F040F9A9B2301D02F03CF90548283869
:1010E000C07800F00301B01D02F034F9BDE8704093
:1010F00002F028B9B707002000E4010841B1012936
:101100000AD0022903D1816841F40001816070474F
:10111000816841F08001F9E7816841F40041F5E719
:101120000A4A914202D1002181617047C1F3130242
:101130008B0101D5C26070474B0101D50261704738
:10114000090101D582607047426070477000F0303D
:1011500030B5082310240422B1F5007F1DD010DC27
:10116000202929D007DC012921D0042922D00829EF
:1011700000D1C46030BD402920D0B1F5807FF9D1C5
:101180000BE00025B1F5004F06D008DCB1F5806F0B
:1011900003D0B1F5006FEDD18561426030BDB1F58E
:1011A000803F0DD0B1F5003FF8D1446030BD054916
:1011B000816030BDC36030BD036130BD046130BDAE
:1011C000436030BD010101003EB5684600F026FADB
:1011D00000208DF8080001218DF809108DF80A0013
:1011E0008DF80B108DF806001D498DF807008DF85D
:1011F000020001F11000897C8DF80310C1788DF890
:10120000041001798DF80510C088164CADF8000067
:101210006946204600F045F901220221204600F0EF
:1012200038F901221146204600F033F90E492046D4
:10123000FFF776FF0C492046891CFFF771FF0B4929
:101240002046FFF76DFF08492046491EFFF768FF5B
:1012500001224FF40441204600F01BF900203EBD5E
:101260006C080020006400400200F0107000F030B4
:10127000094910B588424FF0010101D14C0601E047
:101280004FF08064204604F0BFFD2046BDE81040CA
:10129000002104F0B9BD0000006400402DE9FF47C3
:1012A0000026012119488DF80B608DF80C10DFF82D
:1012B0006090ADF808608DF80D10354634464FF05B
:1012C000040809F1800AC7681AE000BF8DF80A40D7
:1012D00059F82610761C480BADF8000008EBC10148
:1012E000ADF802105AF825106D1C4A0BADF8042019
:1012F00008EBC100ADF80600684600F00BF8641C6E
:10130000BC42E3DB04B00020BDE8F08758080020B1
:10131000C0180020F0B5827A012191402E4A13684E
:1013200043F0010313602C4B1C331C688C431C607E
:10133000294D067B294C0C35A6B92E688E432E60AC
:101340004688C78846EA0746877A04EBC707C7F886
:1013500040660688878846EA0746877A04EBC7070F
:10136000C7F84466067B012E12D12E680E432E600C
:10137000867A056804EBC6064FEA3545C6F840563E
:10138000867A456804EBC6044FEA3545C4F84456EE
:10139000114CC57A241D002D256806D00D4325600B
:1013A0000D4C0589143415B104E08D43F7E7256829
:1013B0008D4325600589012D02D125680D432560E7
:1013C000407B012802D1186808431860106820F09B
:1013D00001001060F0BD00000066004000600040A9
:1013E0000246002053690B424AD0B1F5807F3BD0C2
:1013F00013DC08292ED007DC012926D0022927D0AA
:1014000004293DD1D0682BE0102925D0202926D0F1
:10141000402935D11069102130E0B1F5004F2BD0B3
:101420000BDCB1F5007F22D0B1F5806F22D0B1F591
:10143000006F25D19069702120E0B1F5803F11D077
:10144000B1F5003F1CD15068E5E790680D4915E003
:10145000D06802E0D068DEE7106903210EE0106971
:1014600008210BE05068FBE79069012106E09069D4
:10147000022103E0906900E05068042100F0E4BF1D
:1014800070470000010101008069C0F302100001F3
:101490007047002A426901D00A4300E08A43426152
:1014A000704710B50368002223F00203036003684D
:1014B00043F0010303604FF6FF7300E0521C4468E1
:1014C000E40701D19A42F9D14268D2073ED08A7925
:1014D000012A02683CD022F080020260CA79012A07
:1014E000026838D022F0400202600A7A012A0268BB
:1014F00034D022F0200202604A7A012A026830D0F9
:1015000022F0100202608A7A012A02682CD022F0AE
:1015100008020260CA7A012A026828D022F0040276
:1015200002608A78CC78920742EA04620C7942EA37
:1015300004424C79098842EA0452491E0A43C261B6
:10154000016821F001010160002114E0002010BDBC
:1015500042F08002C1E742F04002C5E742F02002BB
:10156000C9E742F01002CDE742F00802D1E742F0AD
:101570000402D5E7491C4268D20701D09942F9D14B
:101580004068C007E2D1012010BD000010B500EB9B
:101590000113D3F8B04114F004041472D3F8B0412D
:1015A00034D0E408C2F80440D3F8B04104F0020497
:1015B0005472D3F8B44104F00F049472D3F8B441D8
:1015C000240AD474D3F8B841D472D3F8B841240AA9
:1015D0001473D3F8B841240C5473D3F8B841240ED3
:1015E0009473D3F8BC41D473D3F8BC41240A147467
:1015F000D3F8BC41240C5474D3F8BC311B0E937443
:1016000039B1016941F02001016110BD640D146020
:10161000CAE7C16841F02001C16010BD002181719D
:10162000C171017241728172C1728170C1700321F6
:1016300001710221417101210180704730B50246DC
:10164000002093685B0108D49068000101D5012057
:1016500003E09068C00037D5022002EB0012D2F8F8
:10166000803103F00103C2F880310B7A73B3D2F8F2
:1016700080414D681C434B7A43EAC5031C43C2F8C2
:1016800080418B7A03F00F038B72D2F8843123F000
:101690000F03C2F88431D2F884318C7A2343C2F824
:1016A0008431CB7ACC6843EA0423C2F88831CB7BFF
:1016B000096943EA0121C2F88C11D2F8801141F086
:1016C0000101C2F8801130BD042030BDD2F8803154
:1016D0004C7A23430C8843EA4453C2F88031D0E764
:1016E0002DE9F04FFE481A2185B0406CB0FBF1F0B7
:1016F00086B20D20B6FBF0FAFA48FB49B0F91A00A1
:10170000C0F30F100490B1F91020C82042434FF4E9
:101710007A7000EBA2339CB2092303EBA232132AA6
:1017200000D2044689460D46B1F91E0001F00AF9BF
:101730000390B5F9200001F005F90290B5F92200F7
:1017400001F000F9E94B0190D88B4FF4FA7148434E
:1017500040F6FF71B0FBF1F0DFF894C31FFA80F898
:10176000E44DBCF81000E4490090E8880A780709C5
:1017700067F30002C70A67F34102C70867F38202F2
:10178000870867F3C302070B67F30412470867F380
:10179000451260F38612470B67F3C7120A704A7846
:1017A000470A67F30002470967F34102870967F3B5
:1017B0008202070A67F3C302C70967F304122F7A8C
:1017C000BF0867F34512800B60F386124A7093F8E6
:1017D000070110B142F0800001E022F08000487063
:1017E000C4489B46827A887862F341001A461B8976
:1017F000DD0885EA1325ED4365F382009CF800506F
:1018000065F304105D0965F34510DB0A63F3861088
:101810001388DB135B1C63F3C71088709BF84A20A6
:101820002AB1012A07D0022A0AD0032A0DD0CA7889
:1018300022F003020CE0CA7822F00302521C07E0F7
:10184000CA7822F00302921C02E0CA7842F0030236
:10185000A94BCA702833A3F118059A7802F0030245
:10186000012AAA7812D022F01002AA70CA7897072B
:101870000FD020F0080088709F482830407900F091
:101880000300012808D0022809D00BE042F0100222
:10189000EBE740F00800EEE742F0040001E022F040
:1018A0000400C870944F3246791DF87820F09000FB
:1018B000F870381D05F062F9904EB6F9020006F096
:1018C0003BF8B871B6F9040006F036F8F87107F184
:1018D0000806711C3046049A05F050F92246F11CA6
:1018E000B01C05F04BF986486421B0F90400484368
:1018F000800B03F061FA70714246F11DB01D05F0D6
:101900003DF9B9F91000FFF769FAC8214843000C06
:1019100003F052FA287006F1200001240178022712
:10192000B4EB911F03D1A97841F0010105E0B7EBB9
:10193000911F03D1A97821F00101A970437803F028
:101940000301012902D0022904D007E0A97841F05F
:10195000020102E0A97821F00201A970DBF8082059
:10196000A9784FEAD21C6CF38201A97090F802C0EA
:101970005E46CCF3810CBCF1010F03D0BCF1020F29
:1019800003D005E041F0200101E021F02001A97021
:101990008346A046B4EB931F03D1C8B240F0800049
:1019A00004E0B7EB931F02D101F07F00A870554807
:1019B000DFF84091504C417FE878183461F34100E2
:1019C000D10A61F3820096F82A1161F3000031799F
:1019D00061F3C300E87099F80A302979484663F347
:1019E000820133785B115B1C63F3C301530963F31A
:1019F0000411297111166A79491C61F3C3026A71D5
:101A000099F80020E97962F30301C28899F8080087
:101A1000D20B62F38611C00860F3C711E971524618
:101A2000611C204605F0AAF8E11CA01C009A05F0F4
:101A3000A5F8B6F9E800FFF7D1F9C8214843800BB3
:101A400003F0BAF92071307AC109A07961F3C710A7
:101A5000B6F8C8100A0A62F30600A071E171273CCB
:101A6000611C2046039A05F089F8E11CA01C029A2B
:101A700005F084F8611D201D019A05F07FF884F8B7
:101A800006A09BF800005C4620F00C00001D20F032
:101A90003000103020F0C00340338BF800309BF84A
:101AA0000100DFF854A020F00300401C20F00C00DF
:101AB000001D20F0C00240328BF80120A078AAF16E
:101AC0001F0A20F00300401C20F00C00001DA07035
:101AD0008346E07820F0E0014031E17014E000003E
:101AE00038010020D404002040050020A802002076
:101AF000C00A0020100C00208F070020080E0020D4
:101B0000F2050020300E00209AF8000000287DD059
:101B1000F07B00287AD18AF800000AF1170090F8CB
:101B200000C00CF0030CBCF1010F06D090F800C00F
:101B30000CF0030CBCF1020F04D190F800C06CF360
:101B4000010323700378C3F38103012B04D00378CE
:101B5000C3F38103022B06D103784FEA930C237859
:101B60006CF3830323700378C3F30113012B04D0B8
:101B70000378C3F30113022B06D103784FEA131C39
:101B800023786CF3051323700378B8EB931F03D00D
:101B90000378B7EB931F06D103784FEA131C237821
:101BA0006CF387132370437803F00303012B04D0F5
:101BB000437803F00303022B03D1437863F301025C
:101BC00062704278C2F38102012A04D04278C2F3E3
:101BD0008102022A05D142789308627863F3830276
:101BE00062704278C2F30112012A04D04278C2F333
:101BF0000112022A05D142781309627863F30512B3
:101C000062704278B8EB921F05D000E018E142788C
:101C1000B7EB921F05D142781309627863F38712FC
:101C20006270827802F00302012A04D0827802F006
:101C30000302022A04D183785A4663F30102A27098
:101C40008278C2F38102012A04D08278C2F3810231
:101C5000022A05D182789308A27863F38302A270E6
:101C60008278C2F30112012A04D08278C2F30112F1
:101C7000022A05D182781309A27863F30412A270B4
:101C80008278B8EB921F03D08278B7EB921F06D10F
:101C90008278C2F30113A27863F34712A270C2786C
:101CA000D20608D0C27802F01F021F2A03D2C278DF
:101CB00062F30401E170C178490905D0C1784A098D
:101CC000E17862F34711E170017901F00301012924
:101CD00004D0017901F00301022904D101792279AC
:101CE00061F3010222710179C1F38101012904D05C
:101CF0000179C1F38101022905D101798A0821798D
:101D000062F3830121710179C1F30111012904D02A
:101D10000179C1F30111022905D101790A0921795B
:101D200062F3051121710179B8EB911F03D001799C
:101D3000B7EB911F05D101790A09217962F3871167
:101D40002171417901F00301012904D0417901F0A9
:101D50000301022904D14179627961F301026271C0
:101D60004179C1F38101012904D04179C1F3810195
:101D7000022905D141798A08617962F38301617191
:101D80004179C1F30111012904D04179C1F3011155
:101D9000022905D141790A09617962F3051161715E
:101DA0004179B8EB911F03D04179B7EB911F05D171
:101DB00041790A09617962F387116171817901F0D2
:101DC0000301012904D0817901F00301022904D122
:101DD0008179A27961F30102A2718179C1F3810154
:101DE000012904D08179C1F38101022905D18179CA
:101DF0008A08A17962F38301A1718179C1F301118C
:101E0000012904D08179C1F30111022905D1817919
:101E10000A09A17962F30511A1718179B8EB911FCB
:101E200003D08179B7EB911F05D181790A09A17996
:101E300062F38711A171C179E07961F30300E07168
:101E4000434F387800F00F00042801D1FFF720F944
:101E50002078C0F38100012839D1F879010636D500
:101E600000F07F00142832D8A87840F00400A87051
:101E7000384AA978107F8B074FF47F412BD58028F3
:101E800021D3354B00F01F00126853F820000242A6
:101E900019D1B06840F08070B0602D48303880783B
:101EA000C0071CD0B068C00119D52C48406C32283E
:101EB00015D85446BAF802008A46504527D101F099
:101EC0002DFD60800DE0B06820F08070E4E7A87818
:101ED00020F00400CBE7B06820F08070B060AAF872
:101EE0000210A878800702D40020A9F80A003879E7
:101EF000C00701D0A9F80A8099F80A00C107144860
:101F0000A0F14900017812D041F0010111E001F087
:101F1000EDFC40F6B8318842E3D3B068C101E0D5AA
:101F20000005DED4A9F80A80A4F802A0D9E721F0C0
:101F300001010170B168C901017802D541F00201C7
:101F400001E021F00201017005B0BDE8F08F000052
:101F5000BF070020F805002018B70008380100204E
:101F600070B51548006810F0E05F23D0134CD4E939
:101F7000001081421ED004EB001104F5A1608A68B4
:101F800042600A7B827204230372002545720B3083
:101F90000E31FEF7F8F872B66068401C60604028A9
:101FA00000D3656062B60649BDE870400248083853
:101FB000FFF744BB70BD000008640040B814002067
:101FC000C0190020FCB505464FF6FF7600200C46F0
:101FD000ADF8006048F205078DF8040020E000BF6E
:101FE00015F8010B8DF8040001A9084602F070FCF9
:101FF000BDF800009DF8041080EA0120ADF8000053
:102000005FF00000BDF800100A0402D587EA410124
:1020100001E006EA4101401CADF800100828F1DBA0
:10202000641EDDD26946084602F03CFCBDF80000A3
:10203000FCBD00000246002004E000BF12F8013B96
:102040001844C0B2491EF9D27047000070B5144A56
:1020500085B010880024134901940094039420460D
:102060000494138807E0CD8B009E354400950D8BBA
:10207000019E3544019515889D42F4D0401CC0B2A4
:102080008028EED300984111074841808480019850
:102090004111064881830183818205B070BD000033
:1020A00058070020A8020020F2050020D4040020D8
:1020B00030B4104C002003464FF47F42A4F13401A9
:1020C00021F8103024F81020401C1A28F8DB0A4BA5
:1020D000002000BF33F8104021F81040401C1A289F
:1020E000F8DB064806490280012081F8300030BC48
:1020F00003F040BA7C100020180800204C08002093
:10210000DC0E00202DE9F84303F080FAC64DC54BE4
:1021100000204FF47F4105F1340400BF35F8106012
:1021200033F81020964203D025F8102024F8101020
:10213000401C1A28F2DBBD4890F83000012808D076
:102140005FF0000024F81010401C1A28FADBBDE8EC
:10215000F88302F0E1FE208801F0C8FB2988B44E24
:1021600088420AD301F0DAFB2080B24800906B4627
:102170000822B149306809F005F8608801F0B6FB23
:10218000698888420CD301F0C9FB6080A948AA493C
:10219000401C00906B4608220831306808F0F2FFBE
:1021A000A08801F0A3FBA98888420CD301F0B6FBFC
:1021B000A080A048A049801C00906B4608221031E6
:1021C000306808F0DFFFE08801F090FBE988884282
:1021D0000CD301F0A3FBE08096489749C01C009007
:1021E0006B4608221831306808F0CCFF208901F0D6
:1021F0007DFB298988420CD301F090FB20818D481A
:102200008D49001D00906B4608222031306808F08F
:10221000B9FF608901F06AFB698988420CD301F03B
:102220007DFB608183488449401D00906B460822F5
:102230002831306808F0A6FFA08901F057FBA846B6
:10224000A98905277D4D884216D36878052813D2C1
:1022500001F064FBA0816878401CC0B2687005285A
:1022600000D96F7073487449303000906B46082273
:102270003031306808F086FFE08901F037FBB8F8AC
:102280000E10884216D3A878052813D201F046FB19
:10229000E081A878401CC0B2A870052800D9AF70B2
:1022A00064486549313000906B4608223831306807
:1022B00008F068FF208A01F019FBB8F81010884276
:1022C00016D3E878052813D201F028FB2082E8789D
:1022D000401CC0B2E870052800D9EF705548564937
:1022E000323000906B4608224031306808F04AFFD7
:1022F000608A01F0FBFAB8F81210884216D32879E8
:10230000052813D201F00AFB60822879401CC0B274
:102310002871052800D92F7146484749333000906D
:102320006B4608224831306808F02CFF208D01F000
:10233000DDFAB8F82810474688420BD301F0EEFAD0
:1023400020853F483C4900906B460822A031306808
:1023500008F018FF608D01F0C9FA798D88420CD31E
:1023600001F0DCFA608536483349401C00906B462A
:102370000822A831306808F005FFA08D01F0B6FAF8
:10238000B98D88420CD301F0C9FAA08529482A49A1
:10239000503000906B460822B031306808F0F2FEF1
:1023A000E08D01F0A3FAF98D88420CD301F0B6FA62
:1023B000E08520482049603000906B460822B83103
:1023C000306808F0DFFE208E01F090FA398E8842E6
:1023D0000CD301F0A3FA208616481749613000900B
:1023E0006B460822C031306808F0CCFE608E01F0E8
:1023F0007DFA798E88420CD301F090FA60860D4800
:102400000D49623000906B460822C831306808F0F0
:10241000B9FE0C48FFF738F800283FF498AE287052
:1024200095E600001808002048100020DC0E00206F
:102430005C0800200002FF18100F00205008002048
:102440000006FF1800640040024600200A4200D047
:102450000120704730B50E4902880A800C4A438833
:10246000083A13800B1F808818802024151F2C80A9
:102470000020401C80B23C28FBD341F69910088014
:1024800044F64800108046F6480018802C8030BD85
:10249000202C0140114944F648000880091D46F6E9
:1024A00048000880091D41F6991008800B48001F5C
:1024B000018841F02001018009480021A0F868103E
:1024C000A0F86610A0F86410A0F86210A0F86010E0
:1024D000A0F85E100348418181827047182C0140AA
:1024E000A80200204C0000202DE9F04F4C4B4D4835
:1024F0000021DA7A0778802A27F001067CD31C684D
:10250000494B02F01F0253F82220484B14421A682C
:1025100002D042F0200201E022F020029946DFF8CA
:1025200010B11A60444B414D9BF80040DFF804A104
:10253000B3F9043095F84A50022C5ED1D9F808C09E
:10254000CCF3C004CCF30028444556D0374C383C7B
:1025500094F80480B8F1000F06D0B8F1010F0DD047
:10256000B8F1020F4ED120E011054BD5910649D4A8
:102570000121217127F00401017043E0160541D4C7
:1025800096063FD57E073DD44688A6BB4380002BE8
:1025900009DD47F005010170022121712749B1F8D9
:1025A000441001822EE021712CE0C7880FB9002B66
:1025B00016DC077BAF4213D1214FBF895FEA477812
:1025C0000ED45FEA87780BD45FEA427808D55FEAD9
:1025D000826805D5FF0703D115B15FEACC1711D585
:1025E00006704180AAF8001041810182217189F8AA
:1025F0000F108BF8001005E00DE006704180AAF87E
:1026000000104181C3800573500960F3CB22C9F8E3
:102610000020BDE8F08F067041804181F9E700009D
:10262000F8050020C00A002018B70008A802002002
:102630004F0700200C010020F20500203801002087
:10264000100C00202DE9F04F97B000240C940D944D
:102650000E940F9472B6B348816941F400718161A0
:10266000816941F4806181614FF4004003F0AAFB6D
:10267000AD4E00213046FEF755F900213046FEF7F9
:1026800047F90021A948FEF743F9A94F0021384630
:1026900000F0D6F901204FF47041401C8842FCD371
:1026A0003046FEF761FAA148FEF75EFAB9463846B1
:1026B00000F0D2F94FF46020CDE912048DF84540C6
:1026C000012004278DF8440010948DF8507010A953
:1026D0003046FEF7DBFA01231A4605213046FEF7A5
:1026E00026FB0123022206213046FEF720FB0123B0
:1026F000032207213046FEF71AFB012304220F2193
:102700003046FEF714FB484600F0A6F901A800F099
:1027100046FA8548874D4C30CDE902540190049724
:102720008020CDE9054040000790800008902020DF
:1027300009904FF44050CDE90A0401A9484600F041
:1027400011FA01213046FEF7EDF80121484600F06C
:1027500077F901213046FEF7DBF847F23051159446
:102760001598401C15908842FAD301213046FEF797
:102770001DFBADF8004040F2DC584FF40077B34643
:102780001FE0404615941599491C15918142FAD3D2
:1027900029880D9808440D9068880E9908440E9079
:1027A000A8880F9908440F90E8880C9908440C9069
:1027B00001215846FEF7FAFABDF80000401CADF8BA
:1027C0000000BDF80000B842DBD35A490D9808312B
:1027D000C01108830E98A1F11004C01148830F980E
:1027E000DFF854A1C01188830C980AF10202C011CD
:1027F00088806068BAF90050504B0580B2F900C07B
:10280000921CA0F802C0B2F90070921C8780B2F945
:102810000060521FC68092F8008040F6B412B8F1F2
:10282000FF0F21D0A5F5D854263C94420FD2ACF529
:10283000D05CACF5937C944509D2A7F5D857263FD8
:10284000974204D2A6F5D856263E964204D3D8889D
:1028500040F48040D8803BE00D8342884A838288E0
:102860008A83C088888033E0B1F90450A5F5D85533
:10287000263D954214D2B1F91850A5F5D855263DFC
:1028800095420DD2B1F91A50A5F5D855263D95427D
:1028900006D2B1F91C50A5F5D855263D954203D373
:1028A000DA8842F48042DA80DA88520410D40A8B43
:1028B00002804A8B42808A8B82808988C1805546FB
:1028C000504600F0CBFB08222846616800F0DCFB94
:1028D00000215D465846FEF725F800214E46484641
:1028E00000F0AEF800212846FEF712F80F4C002148
:1028F0002046FEF70DF80221C802491C8142FCD394
:102900002846FEF731F92046FEF72EF9304600F052
:10291000A3F8FEF711F80A493C20087062B617B018
:10292000BDE8F08F00100240002401400028014063
:10293000080002403805002000E80108100C0020C3
:102940004C07002010B5FEF749FAC8214843800B18
:1029500010BD000070B5204B40F6C81441F2B70519
:102960005B6C48F6E6065C4305EBA4341B4D7343F1
:102970004EF6F61606EBA333C5E90443D460401ABD
:10298000536110609168884202DA4942884200DC53
:10299000116010684343107E0341906A19189162D8
:1029A000506A814200DD9062916A106A814201DBC7
:1029B000084600E09062A86111684C43117C0C410C
:1029C00008412118B2F91C00884204DBB2F91A0050
:1029D000884200DC08B270BD3801002014010020DC
:1029E00010B54FF40054204600F0ACF8002813D086
:1029F0000A49087840F008000870204600F014F8F2
:102A00000021074800F01CF80648C17E012903D1C7
:102A10000021C1760121017710BD0000920600203F
:102A200044000240140D0020C10002D50249086094
:102A300070470249486070470404024000000240A9
:102A40000029016802D041F0010102E04FF6FE7258
:102A5000114001607047000001684FF6FE7211409E
:102A600001600021016041608160C1603149314AEB
:102A70000839904203D1486840F00F0006E02D4A23
:102A80001432904204D1486840F0F000486070472A
:102A9000284A2832904203D1486840F47060F5E734
:102AA000244A3C32904203D1486840F47040EDE73C
:102AB000204A5032904203D1486840F47020E5E744
:102AC0001C4A6432904203D1486840F47000DDE74C
:102AD000184A7832904203D1486840F07060D5E7D8
:102AE000154A111F904203D1086840F00F0006E01C
:102AF000114A1432904204D1086840F0F000086096
:102B000070470D4A2832904203D1086840F4706043
:102B1000F5E7094A3C32904203D1086840F470401E
:102B2000EDE7054A50329042EAD1086840F470203F
:102B3000E5E700000800024008040240406880B257
:102B40007047000001460020CA0001D5034A00E09A
:102B5000034A12680A4200D0012070470004024074
:102B60000000024030B5036847F6F07293430C6AE8
:102B70008A682243D1E904452C4322438C692243CD
:102B8000CC6922434C6A22438C6A22431A43026076
:102B9000CA6842600A6882604968C16030BD00212D
:102BA000016041608160C160016141618161C16119
:102BB000016241628162704710B5114C8CB00021F6
:102BC0002046FFF73DFF2046FFF746FF0D480090E7
:102BD0000D480021CDE901016420CDE903018020E9
:102BE000CDE905010791089109910A9169462046AE
:102BF000FFF7B8FF01212046FFF722FF0CB010BD00
:102C0000580002400438014000090020F0B540F6A9
:102C1000AA222A49C284838B0C88E31A9BB20F2B09
:102C20000DD309888183037E00213BB1244BB3F986
:102C30000A40244B062C03DA818429E08184F0BD0C
:102C4000214C2478022C02D0002CF5D0F0BD1F4C72
:102C500040F68B27656C1B4CA5F22D16BE42B4F9CD
:102C6000004017D2418B491C89B241836429EDD3BE
:102C700064214183B0F92410914201DA01EB221260
:102C80008284641C20B24FF4007118808842DDDB1E
:102C90001980F0BD41F29416B542FADBB0F9245028
:102CA000002D02DDA5EB221200E000228284418388
:102CB000641E20B218800028EADDF0BD580700200D
:102CC0004C000020580400204F070020380100204D
:102CD00010B50446B0F9020043F699114843811338
:102CE000E06840F26662504301EBA030E060B4F966
:102CF000001043F6991251438A13216940F266632A
:102D0000594302EBA131216105F01CFD6061A188EE
:102D100040F6AB2208444010A0F515415539E06259
:102D2000914205D9A0F5F851FF39521C91421DD2AC
:102D300049F25451884202DDA0F5204002E0A0F59E
:102D4000F850FF38206300EB400040F34F0020852F
:102D5000B4F924104A42904201DA104602E0884257
:102D600000DD0846E083228461848AE0A0F5FE420B
:102D7000FF3A41F255518A4214D8A2F6AA202063A4
:102D800000EB400040F34F002085B4F9242051426D
:102D9000E183884201DA084602E0904200DD1046F5
:102DA000404250E0A0F5D442AA3A8A4215D2A2F697
:102DB000AA20206300EB400040F34F012185B4F9C5
:102DC00024004242E2832084914201DA104602E06C
:102DD000814200DC0846608453E0A0F5AA42543AE0
:102DE00041F256539A4215D2A2F6AB20206300EB73
:102DF000400040F34F002085B4F924104A4290422D
:102E000001DA104602E0884200DD08464042E083D5
:102E1000218419E0A0F5804241F254539A4215D220
:102E2000A2F6AA20206300EB400040F34F0020856B
:102E3000B4F92410E1834A42904201DA104602E0DC
:102E4000884200DD0846208462841AE0A0F52852FA
:102E5000AB3A8A4215D2A2F6AA20206300EB4000CA
:102E600040F34F012185B4F92400E08342422284DB
:102E7000914201DA104602E0814200DC08464042FD
:102E8000A9E7B4F91E0041420948B0F900004143E6
:102E90008913E180B4F9201049424143891321810B
:102EA000B4F92210494241438813608110BD0000EB
:102EB0005804002001210176704770471548164AD2
:102EC0004FF480410078042821D002F13C03D08ADD
:102ED0009B88C01A00B22F2801DD001108E00028ED
:102EE00001DD002007E00D4B984201DA184602E0B0
:102EF000402800DD40209389184400B2884203DC5A
:102F000040F26661884200DA0846908170479181FC
:102F1000704700004F070020D4040020C0FEFFFFD0
:102F200038B54B484B4902880B889A1A92B20F2A3F
:102F300071D30988484C01804FF0FF01E2884FF4BB
:102F40007A7355044FF4967002D51622009103E06F
:102F5000950403D515220091014670E0D50402D5F1
:102F600014220091F8E7150502D513220091F3E72A
:102F7000550502D512220091EEE7950502D51122E2
:102F80000091E9E7D50502D510220091E4E7150686
:102F900002D50F220091DFE7550602D50E220091DF
:102FA000DAE7950602D50D220091D5E7D50602D5C0
:102FB0000C220091D0E7150702D50B220091CBE738
:102FC000550702D50A220091C6E7950702D50922C6
:102FD0000091C1E7D20702D008220091BCE7228904
:102FE000550702D507220091B6E7950702D50622BC
:102FF0000091B1E7D20702D005220091ACE7A27A96
:10300000D20702D004220091A6E7A289D40603D5F4
:1030100003220091A0E719E0140702D502220091D3
:103020009AE7540703D4940701D4D20702D00122AF
:10303000009191E70020034602460146009003F00C
:10304000B9FCBDE838400248FDF79EBF38BD00001E
:10305000040C002058070020100C002070B5054615
:10306000002472B600F0BCF9252000F031F92846A2
:1030700000F034F9042801D04FF0FF3400F062F979
:1030800062B6204670BD00002DE9F04700251746C6
:10309000894680462C4672B600F0A2F912E000BFC5
:1030A00059F82460352000F013F93146404600F00D
:1030B0006DF9042802D04FF0FF3506E0641C08F1DA
:1030C0000408E4B2B4EB970FEAD300F03BF962B620
:1030D0002846BDE8F0870000F0B559485949828874
:1030E0000B889A1A92B29C2A64D309888180564927
:1030F0000A880146002A0B7843F0020156D1164691
:10310000524A1C0715680246127822F0020274D552
:103110004F4C0746E4887F785FEA845C02D547F02D
:10312000010701E027F001074770A704477802D59F
:1031300047F0020701E027F002074770670401D457
:10314000E70703D0477847F008074770640603D5C0
:10315000447844F0040404E01C0603D4447824F0CA
:1031600004044470EC0450D4354C9A07247824F0BD
:10317000100423D4324D42782F7A2D78012A45F05D
:10318000100514D0022A16D02D4C042AA47804F17C
:10319000010C0CF0FF0C13D0072A25D0032A23D0F2
:1031A000052A21D0062A1FD021F0100142E0B907DC
:1031B00002E00570F0BD39070029FADB0470F0BDAC
:1031C000FA0601D41A060AD50170022C04D280F83E
:1031D00002C0BCF1020FF2D341F080012AE021F0DD
:1031E000100101708670F0BD877A7F06F7D5032C39
:1031F00004D8017080F802C0F0BD0FE05107D8D5A7
:103200001906D6D443F0800114E002704178CB0750
:1032100001D18907F0D522F010010BE0E9040BD4AD
:103220009907E9D4818AC82902D2491C8182E3E73F
:1032300043F00A010170DFE702708682DCE70000DC
:1032400020070020580700205A070020A80200206D
:10325000100C002070B51148114C4FF00005C088CB
:10326000810503D4410601D4C00515D54FF4806112
:103270000C4800F02BFB68B9A08840F6B8318842B2
:1032800001D2401CA08080B2B0F57A7F01D301202A
:10329000607070BDA58070BD6570FBE7100C0020EC
:1032A00070070020000C0140084946F668000880BD
:1032B000091D0880091D41F6DD5008800348001FE4
:1032C000018841F02001018070470000182C014066
:1032D0000149C860704700000020024070B50D4EE3
:1032E0000546304600F088F8042811D10A4C2069C0
:1032F00040F0020020616561206940F040002061DB
:10330000304600F079F8216941F6FD7211402161E3
:1033100070BD0000FFFF0F0000200240084904209C
:10332000CA68D20701D001207047CA68520701D588
:1033300002207047C968C906FBD50320704700000A
:10334000002002400248016941F08001016170479C
:1033500000200240F0B506464FF6FF770D4638468E
:1033600000F04AF804280DD1074C206940F0010014
:1033700020613580384600F03FF8216941F6FE7241
:1033800011402161F0BD0000002002402DE9F8410C
:10339000064600204FF6FF7700900D46384600F0B5
:1033A0002BF8042817D10D4C206940F00100206152
:1033B0003580B846384600F01FF841F6FE770428FD
:1033C00006D1B61C280C00963080404600F014F858
:1033D000216939402161BDE8F881000000200240E8
:1033E0000348024941600349416070472301674532
:1033F00000200240AB89EFCD00B50346FFF78EFFFA
:1034000003E000BFFFF78AFF5B1E012803D0002BFB
:1034100000D1052000BD002BF4D1FAE710B5C28819
:1034200000210AB1032206E002890AB1022202E069
:10343000428912B10122027000E0017004784FF459
:10344000804344F6206244B1012C06D0022C07D000
:10345000032C01D14180818010BD4380828010BD4A
:1034600041F23331418040F6B731F4E7401A106041
:103470009168884202DA4942884200DC1160516951
:103480001068137E41431941936A0B449362516A59
:103490008B4200DD9162936A116A8B4200DA91627D
:1034A000D168936A4143107C01410341B2F91C0089
:1034B0001944884204DBB2F91A00884200DC08B2E1
:1034C00070470000054920B1086940F0800008619C
:1034D0007047034848600348486070470020024036
:1034E00023016745AB89EFCD06494FF47A70CA686E
:1034F000D20705D0401E0004000CF8D1FF20704711
:1035000000207047002002400E4A0320A2F14C0127
:1035100082F83E000020C8800B490886C862C88334
:103520000884488490620948016DB1F5206F01DB81
:10353000A3219162807A002802D0906A4042906272
:10354000704700004C00002040050020380100209A
:10355000F0B53D4988894A89801A80B20F286AD31C
:1035600088894881CA8939480B3A272A26D28A781D
:1035700022BB8268384B42F480728260344A374CF6
:10358000374D12785607334A0AD4364E368816809D
:10359000354A12881A80354A12882280344A09E056
:1035A000344E36881680344A12881A80334A12887C
:1035B0002280334A12882A8001228A70314A0021EF
:1035C000314B82F84D1019469A7F304D0968802A98
:1035D00032D302F01F0255F8222011422CD082680B
:1035E00022F48012184E8260123614461215B778F3
:1035F000521C62F38617264AB77093F816C01778E4
:10360000BCF1800F27F0020608D30CF01F0C55F810
:103610002CC011EA0C0F01D147F0020616701A7E79
:10362000802A0DD302F01F0255F82220114207D143
:1036300044F400218160F0BD826842F48012D1E739
:1036400024F40021F6E700004C070020A802002027
:1036500038010020CC040020CE040020D00400203B
:10366000D2040020BC040020BE040020C0040020BE
:10367000C2040020C4040020C6040020C8040020A6
:10368000CA040020680E0020F805002018B70008C2
:10369000D404002070B5214881890289891A89B231
:1036A0000F2932D381891E4D1E4C0181697A22680F
:1036B0001D4E42F00400802908D301F01F012B6841
:1036C00056F821100B4201D122F004002060FFF7D0
:1036D000C1FDA87B802819D300F01F00296856F887
:1036E0002000014212D1206820F002002060E87A18
:1036F00080280FD300F01F00296856F820000142EF
:1037000008D1206820F00800206070BD206840F0DB
:103710000200EBE7206840F00800F5E74C070020C6
:10372000F8050020A802002018B7000830B50446AC
:1037300000204FF40043024640EA030101FB01F57B
:10374000A54200D80846521C5B0812B2102AF3DBCF
:1037500030BD0000F0B51D4C1B4A4FF0010C94F831
:103760003B5094F80AE0144692F83C3094F8384004
:103770002B43651CEEB2154D95F83D700025BEF14A
:10378000FF0F0AD0BEF1000F06D18B4213D1557046
:103790000C2C01D282F83860F0BD834202D182F84D
:1037A00001C0F5E78B42F7D15570B80709E000BFBB
:1037B00082F83850F0BD8342FCD1F84382F801C052
:1037C00080070028F4D0F0BD5C0400203801002000
:1037D000F0B5CA78002502F00F03D20601D58A7829
:1037E00013430A784FF00F0E12F0FF0F4FF0010253
:1037F0001CD004680F8802FA05F63740B74211D191
:103800004FEA850C0EFA0CF724EA070703FA0CF4CA
:103810003C43CF78282F02D0482F02D002E04661E7
:1038200000E006616D1C082DE4D304600C88FF2CB9
:103830001ED944685FF0000606F1080702FA07F592
:103840000F882F40AF420FD14FEA860C0EFA0CF7CB
:10385000BC4303FA0CF73C43CF78282F00D14561D5
:10386000CF78482F00D10561761C082EE4D3446040
:10387000F0BD0000F0B5144C002801DAE36900E067
:103880006368420D120185B2C0F301579540C0F341
:103890000346032F05D0C2020AD50322B240934348
:1038A00007E023F07062636823F07063636002E0F6
:1038B000AB4343F0706201B12A43002801DAE261B0
:1038C000F0BD6260F0BD0000000001400246002033
:1038D00092680A4200D0012070474161704701613F
:1038E00070470AB101617047416170474FF6FF624E
:1038F000B0F57F4F04D0911C884203D1002070475F
:103900001046704704490988814201D3081A01E032
:10391000101A084480B270479808002001480088B7
:1039200070470000980800200F4A104B92F838109A
:103930005B5C834201D1012004E00D4B5B5C834260
:1039400003D1002082F83A0070470A4B5B5C834247
:1039500001D18120F6E7084B595C814201D18020DA
:10396000F0E70320EEE7000038010020D0BB00089C
:10397000E2BB0008D6BB0008E8BB00080A4810B547
:1039800001784FF000024C0708494FF0FF038968A7
:103990004FEA017105D5002901DA827210BD8372E8
:1039A00010BD0029FBDBF8E738010020A802002049
:1039B000F0B5194E194C0022E31CA6F1060CB75CB9
:1039C000A518ED78FF5C0D430F43BD421FD01CF8D6
:1039D0000270FF5C0F43BD4219D015460023A618A4
:1039E000F6780E43C6545B1C1CF80220DBB2062B93
:1039F000F5D3C17881700179C17000214218491C4A
:103A000015711CF80550C9B20629F7D3F0BD521C38
:103A1000D2B2032AD3D3F0BDAAB200085C040020BE
:103A200010B502460021064B06205C1864789442CB
:103A300000D10846491CC9B20629F6D310BD0000C2
:103A4000380100200548D0E900218A4202D14FF018
:103A5000FF30704700EB011080687047B010002005
:103A600070B5164C05464FF0FF36D4E90010814280
:103A700021D004EB001080686860606804EB0010DF
:103A8000007B00F00F02AA7204202872606804EB29
:103A9000001105F10B000E31FCF775FB72B6606882
:103AA000401C6060402801D30020606062B6A87AA4
:103AB00008B1002070BD304670BD0000B01000207D
:103AC00070B526484FF000028078C10724483FD0E7
:103AD00024498988E1BB2449234B4FF4FA65496C9A
:103AE000B3F87630A94231DD90F84A1071B31F491E
:103AF000C9790C062AD501F07F015A2926D290F8FF
:103B00002B11491CC9B280F82B11C8291ED380F88B
:103B10002B21D0F83041014604F1640691F82C11B4
:103B2000B34203DD052908D2491C01E041B1491E19
:103B300080F82C11C9B2052902D3012180F82A117D
:103B4000191B074C383C2163C0F83031AB4203D21B
:103B500080F82A2180F82C2170BD00009F070020EA
:103B6000A8020020F205002038010020BF07002035
:103B70004FF42032C260002181620E22028241F2A3
:103B800062024261082202834FF4604242838183D1
:103B90004FF07842C0E9082140F6C4110180704717
:103BA000B0F90010B0F90220891A41604269037E21
:103BB0004A431A41836A13448362426A934200DD96
:103BC0008262836A026A934200DA8262C268836A0E
:103BD0004A43017C0A410B41D118B0F91C208A42AA
:103BE00001DA10467047B0F91A008842FADC08B2D0
:103BF0007047000010B514481449B0F894200B88A1
:103C00009A1A92B2B2F5437F1DD90988A0F8941090
:103C1000B0F8921020F8601F002242860C480D4C2C
:103C2000C2888280C180C38983812489891AA4B211
:103C3000C4818160E11A0161074A818AC182928A46
:103C40008282511A816110BD38010020580700207E
:103C5000300E0020400500204C00002009480A4991
:103C6000B0F8B2200B889A1A92B241F684639A4255
:103C700006D3098820F8B21F418881800021418045
:103C80007047000038010020580700200D480178D7
:103C9000C90702D00C49098801E04FF6FA71416664
:103CA000094901201039088007482438018841F06B
:103CB0000101018004481838018821F018010180B1
:103CC0007047000038010020240400400A49D1F860
:103CD000982012B1521EC1F8982031F8922F521C30
:103CE00021F81A294A6A521C4A628A8F521C8A8712
:103CF00001F8400C70470000380100201CB52D4829
:103D000090F83B3090F83C20934252D000248DF83C
:103D1000044053408DF800309DF800300122012B03
:103D200008D09DF80030022B09D09DF80030042BFC
:103D30000AD00DE01F498DF80420443108E01D49E8
:103D40008DF80420463103E01A498DF804204831EB
:103D50009DF80420012A2CD190F83D309DF80040B8
:103D6000154AA34217D090F83E309DF800402342F8
:103D700008D0B0F84C30A0F84A300B881488E31A09
:103D8000A0F84C3090F838302BB1B0F8403014889F
:103D9000E31AA0F8423012880A80A0F8402010F8F8
:103DA0003E1F9DF80020114300F801199DF80010F6
:103DB00001701CBD5C0400205807002070B5354D13
:103DC0004FF480712846FFF781FD8400802128464A
:103DD000FFF77CFD44EA400440212846FFF776FDCA
:103DE0000443E1B22C4C94F878508D4250D04D40B1
:103DF00084F87810012D03D0022D01D0042D47D175
:103E000094F87C00A84384F87C0094F87B20AA42B4
:103E10000FD084F87B5094F87A2001238B401A420B
:103E200007D11A4384F87A2094F87910491C84F851
:103E3000791094F87910042928D330B1012811D0D1
:103E400002280FD004280DD012E01448C18821F0B8
:103E50004001C1802078002184F83B1020F06000F0
:103E6000207005E0217841F02001217084F83B00AA
:103E70000B4994F83B0091F82720904204D081F838
:103E8000270008492020087000F00EF884F85450EC
:103E900070BD00000010014038010020100C00200F
:103EA000680E00204C07002070B50E4D4FF4807155
:103EB0002846FFF70BFD840080212846FFF706FD0A
:103EC00044EA400440212846FFF700FD0443064829
:103ED000072100F8784F0171002141708170C17095
:103EE00070BD0000001001403801002070B534485A
:103EF00090F83A10CA43920761D001F0030280F8AB
:103F0000392090F83D305B061B0E80F83D30012AC9
:103F100001D0812A02D15B1C80F83D300278D207A3
:103F20004DD0DBB203F00102C3F34004A24246D1FC
:103F3000B0F856400025641CA0F85640204CA0F86C
:103F4000585090F83E60A47AB24202D080F83E20E9
:103F50000DE0A607B6EB837F02D080F83F5006E065
:103F600090F83F30642B02D25B1C80F83F3090F811
:103F70004030642B0CD25B1CDBB280F84030022B4B
:103F800006D204F00103934202D1022280F84020BD
:103F9000012901D0002912D190F83820416E00EBA0
:103FA000820291610163D0E906121144D0E908232D
:103FB0001A441144826A1144C26A1144416370BDBB
:103FC00038010020FEE700002DE9F04F00BF00207F
:103FD0009E4E9F4AA6F51271A6F5BE79A6F1440B36
:103FE00006F1440E804601F5E074A1F1780301F575
:103FF000457A1D5C15F0C00706D0402F51D0C02F68
:1040000077D0802F76D004E115F01F0504D0154439
:1040100040F080072F7201E082F80880012826D046
:10402000022824D0032822D0042820D008281ED01B
:1040300010281CD0874D55F820C0DCF8005054F8EB
:1040400020703D40CCF80050824D55F820C0DCF87F
:10405000005056F820703D43CCF800501D5CAD0672
:1040600059F820502F6813D53AF810C03EE051F8A7
:1040700020502F6854F820C007EA0C072F6051F831
:1040800020502F6856F820C047EA0C072F60E5E75C
:10409000DFF8B8C10CF1F00C5CF820C007EA0C079F
:1040A0007EE015F01F0504D0154440F080072F7204
:1040B00001E082F8088001281DD002281BD00328C7
:1040C00019D0042817D0082815D0102813D0614D16
:1040D00055F820502F6854F820C007EA0C072F60CD
:1040E0005C4D55F820502F685BF820C047EA0C075C
:1040F00056E00BE056E051F820502F6854F820C0ED
:1041000007EA0C072F6051F82050ECE715F01F0567
:1041100005D0154440F0800785F8217001E082F851
:104120002180012825D0022823D0032821D004286B
:104130001FD008281DD010281BD0464D55F820C090
:10414000DCF8005054F820703D40CCF80050414D50
:1041500055F820C0DCF800505EF820703D43CCF8E4
:1041600000501D5CAD0615D53A4D3AF81070CC35AF
:1041700014E051F820502F6854F820C007EA0C07CB
:104180002F6051F820502F685EF820C047EA0C07D6
:104190002F60E6E72D4D3AF81070E03D55F82050BD
:1041A0002F6036E015F01F0505D0154440F080075C
:1041B00085F8217001E082F82180012830D00228A2
:1041C0002ED003282CD004282AD0082828D0102844
:1041D00026D0204D55F820C0DCF8005054F820704F
:1041E0003D40CCF800501B4D55F820C0DCF8005085
:1041F000164F883757F820703D43CCF800501D5CAF
:10420000AD06B1D4114F3AF81050E03F57F8207086
:104210003D60401CC0B21128FFF4EBAEBDE8F08F4A
:1042200051F820502F6854F820C007EA0C072F607F
:1042300051F820502F68DFF814C00CF1880C5CF89E
:1042400020C047EA0C072F60D9E70000A4B9000896
:10425000F8050020A0B700084FF40771C1824FF4A1
:104260005861018340F6145181837047F0B5C48AC8
:10427000B0F900608681B0F90250C581B0F9043010
:104280000227002101220382AB4204DBB54202DD9A
:10429000C78042810CE0B34204DBAE4202DDC7803E
:1042A00041811CE09D4205DBB34203DDC2804781B2
:1042B000018115E0B54204DB9E4202DDC2804181EE
:1042C00005E0AE4205DB9D4203DDC18042810781EE
:1042D00006E09E4204DBAB4202DDC18047810281E1
:1042E000C388458900EB430700EB4505BB89AE89D0
:1042F0009B1B0FFA83FEA0F812E00689AB8900EB46
:10430000460CBCF80CC0A3EB0C038382B0F9183048
:10431000B7F90CC0A3EB0C0CB4EB4C0F04DA80F82B
:104320002010A3F1A10113E0A64503DD80F82010C1
:10433000B9890BE026B1012E04D0022E10D004E082
:10434000062100E0052180F82010A989091B6D31A4
:10435000418309B2B1F5586F04DB5B1E438304E06F
:104360000421F0E7002900DC4283418B8183F0BD0A
:104370000B49002288760A62CA614A62094A32F908
:10438000103002EB40028B62B2F90220CA62064A88
:1043900032F810000882A1F86000A1F862007047AE
:1043A000F0010020FABB0008EEBB00082DE9F05F29
:1043B000FD48FE4982880B889A1A92B20F2A47D389
:1043C00009888180FA498346FA4D0888FA4FDFF858
:1043D000EC934FF00108002678B3401E0880EE737E
:1043E000EE6249462868B1F90210430742F6AA2254
:1043F00018D4FB8843F40053FB8099F800309B07E6
:1044000009D5AB6823F08003AB60A5F8806085F820
:10441000826085F88360C30404D485F8F480C5F80D
:10442000F06003E085F8F460430707D4914205DBB0
:1044300085F8F880A5F8F66004E010E085F8F860EB
:10444000430703D4914201DBC00703D085F815610F
:10445000BDE8F09F85F81581A5F81661F8E7B5F875
:104460001C0143F69821884202D2401CA5F81C0189
:1044700002F0B6FADFF848A39AF8500010B1FEF740
:1044800033F805E0C8481838017821F001010170BF
:10449000FFF716FB00F032FACA4841F26802416C9D
:1044A0004FF40060914201DBC74A04E0B1F57A6F36
:1044B00002DAC54A121D1060C148DFF8F8A20A24CA
:1044C00090F85100DFF804C3C007AAF1380A38D0C9
:1044D0009CF80E00802802D32878800705D5BC48B8
:1044E0000078C20601D4800627D5EA7B8AF8092025
:1044F00099F80030AC4A23F00203183A89F80030EA
:1045000056801378504623F001031370BA7952068F
:104510000FD4C289B2F5FA7F03D2521CAAF80E203A
:104520000FE040F63C70814201DD002466E0042487
:1045300064E00024AAF80E6060E08AF80560AAF83A
:104540000E60A868020501D5082457E09C4A92F83D
:104550003FE05FEACE7246D0EA7B8AF809209CF8F9
:104560000930802B44D39B4B9B781B0640D52B787E
:104570005B0731D4FB889B0404D500BF20F02000EA
:10458000A86030E0884B40F02000183B5E801C782B
:1045900024F001041C70A8609CF8170080280BD33D
:1045A00000F07F044FF00040DCF80030E0400342B0
:1045B00002D185F8048000E02E712879C00702D16D
:1045C0005FEA8E7005D50324032A17D08AF80C8081
:1045D00014E00024EE6211E020F02000A860F888CA
:1045E00020F40050F88095F82A01012805D005E054
:1045F0002A6842F004022A60C0E7092408B276491A
:1046000003F0D2FB6B49754DCA6A50438013A1F881
:10461000E8000A2C7ED16F488078800602D5FCF72E
:1046200053FC09E063488168CA0502D521F00801FE
:1046300001E041F0080181605E484FF400546200DF
:1046400090F84A8042F6CC4142F26663B8F1010F1D
:104650001ED0B8F1020F30D02978DFF884C1B8F14C
:10466000030FC1F381013BD043F6FE7801293ED010
:1046700002293CD0A0F81821A0F8482047F23C318C
:10468000ACF800104E4991F87010012932D03FE08B
:1046900095F800C0CCF3810CBCF1010F07D0BCF140
:1046A000020F07D0A0F81811A0F84810EAE7A0F808
:1046B0001831F9E7A0F81841F6E795F800C0CCF3F7
:1046C000810CBCF1010F08D0BCF1020F05D0A0F89D
:1046D000182100BFA0F84820D4E7A0F81811F9E786
:1046E000A0F81821A0F8482046F65471C8E7A0F8B1
:1046F0001881C1E72978C1F38101012911D002296C
:1047000012D041F6E121A0F8181100BFA0F84830FE
:10471000254900E06DE018390B78DB0707D00B8ADC
:1047200007E0A0F81831F1E7A0F81841EEE7B9F872
:104730000430ABF8123019B2B0F948305943C1F324
:104740008F335146AAF81E30934200D9CA83254AB6
:104750001278D20605D5CB8B41F23332934200D288
:10476000CA838268C2F3C003C2F30024A34205D106
:10477000CC8B41F699139C4200D9CB831A4B9B7882
:10478000DB0707D0D20105D4114A127802F00F02DC
:10479000032A00D0CE83BAF81E10C162002927DD9B
:1047A00012480224067024E0D80A0020580700208E
:1047B0005A070020A8020020100C0020F20500205B
:1047C000680E002038010020100C0140F805002080
:1047D000BF0700209F070020F4B10008D404002088
:1047E00030010020200700208F0700206C070020E8
:1047F00000249BF81A0028BB022C15D014B32648BD
:1048000001788B0608D5BB795B0605D5234B1B7851
:10481000DB0963F386110170F88820F40060F880EA
:10482000B9F8041039B109E0288F0028E7D143F620
:1048300098202887E3E720F08000F88080B220F0FD
:104840002000F8801448406C4E281FDBFB881806B7
:104850001CD5BAF81C104FF4FA75491C89B25046A1
:10486000AAF81C10A94201D9858301E0A94207D307
:10487000B9F8041021B9AAF81C6023F08000F88070
:1048800099F8001021F0020189F8001004488BF813
:104890001A40C473DCE50000380100202007002026
:1048A000A802002070B500230C8863F30F020125D5
:1048B00005FA03F6344206D0C3F10F0605FA06F1F5
:1048C000114361F30F025B1C102BF1DB028070BD02
:1048D00070B500230C7863F30702012505FA03F68F
:1048E000344206D0C3F1070605FA06F1114361F31D
:1048F00007025B1C082BF1DB027070BDF0B520488D
:1049000090F866101F480129836823F4006234D1AF
:104910001D49CE88740630D41C4D1F054FF000048D
:10492000B5F9025020D41A4A526C642A11DC40F6C0
:10493000386295420DDAB2040BD40278520710D4D3
:10494000B0F8D82040F6B835AA4203D2521CA0F8DD
:10495000D820F0BD43F400628260D001F9D44C81CC
:10496000F0BDA0F8D840F0BD41F2CD039D42FADD84
:10497000897AC907F7D18260F3E78260F0BD000051
:10498000680E0020A8020020100C0020F205002074
:1049900038010020F0B5364D364F044695F83B00FF
:1049A00097F83B1023780843EE1C6278834205D1C8
:1049B000E0781146FEF7CEFE207908E094F802C0B8
:1049C00084450CD1E1781046FEF7C4FEE07905F885
:1049D0002F0F2878805D6870287BE877F0BD8242D1
:1049E0001DD161461846FEF7B5FE95F84E1095F8B4
:1049F0003B00814207D1B97A09B1A17900E0617920
:104A000085F82F101EE06978012901D0A17922E0F4
:104A1000617927E0297841F00401297012E0E178FA
:104A20008142DBD119466046FEF794FE95F84E10A0
:104A300095F83B0081420AD1B97A09B1617ADFE782
:104A4000217ADDE715F82F1F895D6970C5E7697860
:104A5000012906D0617A85F82F10B97A0029F1D1A1
:104A6000D8E7217A85F82F10B97A0029EAD0D1E762
:104A70005C040020380100200B48017821F002017D
:104A800000F8381B002100F818194177817733218D
:104A90008185418508214184012100F81F1C0348BC
:104AA00080F83910704700005C04002038010020B5
:104AB0000D4900B50B4851F8012F40F8032F8988A4
:104AC0008180084801210930FEF772FF0548022164
:104AD0001330FEF76DFF034804211D305DF804EB31
:104AE000FEF766BF5C04002038010020094944F647
:104AF00048000880091D46F648000880091D41F25B
:104B0000111008800348001F018841F02001018036
:104B100070470000182C01402DE9F041654C664BB0
:104B20000025A0780126644A103305287ED2DFE8EC
:104B300000F00313113E1100108820F001001080D6
:104B40001D805E480580001F0580001F0580FFF75F
:104B5000CDFFA670BDE8F081584941F6CC401C3924
:104B60000880564945F6580024390880091D46F644
:104B70005800088051492020283908800020401C16
:104B8000C0B27328FBD3FFF7B1FF4B4984F85C50E8
:104B90002C3147F6906008804748143006801D800D
:104BA000108840F0010010800220A070D2E70021A0
:104BB0005FF0010004EB410204EB4003B2F8502027
:104BC000B3F850309A4200D20146401CC0B20628C9
:104BD000F0D33B48405C84F83900FFF74DFF1D20BF
:104BE00000F0B8FD00F074F8364E37484FF480718D
:104BF00096F83B20012A04D0022A1AD0042A2ED08B
:104C000044E08046FEF762FE870080214046FEF7C2
:104C10005DFE47EA400740214046FEF757FE074346
:104C200047F0010084F83B00224800E03AE00930F8
:104C30002AE08046FEF74AFE870080214046FEF7C4
:104C400045FE47EA400740214046FEF73FFE074346
:104C500047F0020084F83B001648133014E0804609
:104C6000FEF734FE870080214046FEF72FFE47EA1C
:104C7000400740214046FEF729FE074347F0040065
:104C800084F83B000B481D3003F08AFB94F82F009A
:104C900086F838001D2000F073FD0420A0700B483A
:104CA000057057E7108820F0010010801D80A57066
:104CB00050E700005C040020000800403C2C01404C
:104CC000B0B2000838010020001001404F0700205A
:104CD0002DE9F041354C14F82F0F354DE0724FF4AB
:104CE000807739462846FEF7F1FD86008021284668
:104CF000FEF7ECFD46EA400640212846FEF7E6FDB9
:104D00000643207BF1B22F3C814215D084F83C0051
:104D100039462846FEF7DAFD860080212846FEF750
:104D2000D5FD46EA400640212846FEF7CFFD064362
:104D300084F83B60FEF7E2FF1E4D95F83B0001282A
:104D400027D0022828D0042829D0184894F83B10EE
:104D50002730085C04F8300F14F80109FEF760FEF4
:104D600004F82F09A87A00B10120607001F0E0FE7C
:104D700094F84E0094F83B10884206D094F838001E
:104D8000062802D2401C84F8380084F84E10BDE892
:104D9000F0810648093004E00448133001E003487C
:104DA0001D30BDE8F041FFF7F5BD00005C040020B8
:104DB0000010014038010020FF2801D9FF20704772
:104DC000C0B270472DE9F0414A4991F87200AA2813
:104DD00074D191F87300552870D1474C00200A5CBB
:104DE0002254401CC0B27428F9D3444E2069C6F83E
:104DF0000100A08AA6F80500D4F81600F060D4F8E7
:104E00001A003061D4F81E001234706103F06EFA9B
:104E10003B49608A888103F083FA207D123CC007F9
:104E2000307802D040F0040001E020F00400354961
:104E300030704FF480400861334D14F8280F334927
:104E400085F82000608B6880A08BA880E08BE880CC
:104E5000208C2881608C688194F8240081F8D60029
:104E600014F8010C86F83B000027C6F89C70FFF789
:104E70001FFE2748A18E0183E18E4183218F81830C
:104E800094F84210283C012908D0022901D00329B6
:104E900009D0297821F00C01083107E0297821F0A8
:104EA0000C01091D02E0297841F00C01297094F8E9
:104EB000642018491AB101224A8101E00EE04F81B5
:104EC00094F8701001290BD094F86D1059B1012994
:104ED0000CD04FF4805100BFA0F87610BDE8F081EF
:104EE00044F21C71F8E74FF40051F5E741F25551D7
:104EF000F2E7000000FC0008680E002038010020E6
:104F00004C000020080E0020D4040020A80200203D
:104F100040050020100C002010B5FCF7E1FBFE4816
:104F2000FE4AFF49807AC00703D0887820F001004C
:104F300005E09078800703D0887840F00100887001
:104F4000F8480B7803704B7843708B788370CB787C
:104F5000C3700B7903714B7943718B798371C97974
:104F6000C171EF49083109780172ED49083149787A
:104F70004172EB49083189788172E9490831C97871
:104F8000C172E749083109790173E5490831497966
:104F90004173E349083189798173E1490831C9795D
:104FA000C173DF49103109780174DD491031497846
:104FB0004174DB49103189788174D9491031C9783D
:104FC000C174D749103109790175D5491031497932
:104FD0004175D349103189798175D1491031C97929
:104FE000C175CF4918310B7803764B7843768B78AF
:104FF0008376CB78C3760B7903774B7943778B79BC
:105000008377C979C177C6490F39097880F82010AC
:10501000C3490F39497880F82110C1490F3989787F
:1050200080F82210BE490F39C97880F82310BC4996
:105030000F39097980F82410B9490F39497980F876
:105040002510B7490F39897980F82610B4492031E5
:105050000B7880F828304B7880F829308B7880F8EE
:105060002A30CB7880F82B300B7980F82C304B79B4
:1050700080F82D308B7980F82E30C97980F82F1088
:1050800000F1D001097880F8301000F1D0014978A2
:1050900080F8311000F1D001897880F8321000F1E9
:1050A000D001C97880F8331000F1D001097980F877
:1050B000341000F1D001497980F8351000F1D001A9
:1050C000897980F8361000F1D001C97980F837105D
:1050D00000F1D001097A80F8381000F1D001497A46
:1050E00080F8391000F1D001897A80F83A1000F187
:1050F000D001C97A80F83B1000F1D001097B80F81B
:105100003C1000F1D001497B80F83D1000F1D00146
:10511000897B80F83E1000F1D001C97B80F83F10F8
:1051200000F1D001097C80F8401000F1D001497CE9
:1051300080F8411000F1D001897C80F8421000F124
:10514000D001C97C80F8431000F1D001097D80F8BE
:10515000441000F1D001497D80F8451000F1D001E4
:10516000897D80F8461000F1D001C97D80F8471094
:1051700000F1D001097E80F8481000F1D001497E8D
:1051800080F8491000F1D001897E80F84A1000F1C2
:10519000D001C97E80F84B1000F1D001097F80F862
:1051A0004C1000F1D001497F80F84D1000F1D00182
:1051B000897F80F84E1000F1D001C97F80F84F1030
:1051C00000F1F0010B7880F850304B7880F85130C6
:1051D0008B7880F85230CB7880F853300B7980F898
:1051E00054304B7980F855308B7980F85630CB7934
:1051F00080F857300B7A80F858304B7A80F8593065
:105200008B7A80F85A30CB7A80F85B300B7B80F851
:105210005C304B7B80F85D308B7B80F85E30CB7BE5
:1052200080F85F300B7C80F860304B7C80F8613018
:105230008B7C80F86230CB7C80F863300B7D80F80B
:1052400064304B7D80F865308B7D80F86630CB7D97
:1052500080F867300B7E80F868304B7E80F86930CC
:105260008B7E80F86A30CB7E80F86B300B7F80F8C5
:105270006C304B7F80F86D308B7F80F86E30C97F4B
:1052800080F86F10264950310B7880F870304B78D9
:1052900080F871308B7880F87230CB7880F873307A
:1052A0000B7980F874304B7980F875308B7980F801
:1052B0007630C97980F87710117880F880105178AD
:1052C00080F88110917801F0030180F88210117943
:1052D00080F88310517980F88410917980F88510D6
:1052E000D17980F88610117A80F887100C4938310E
:1052F0000A7802F0030280F888204A7880F8892032
:105300008A7880F88A20CA7880F88B200A7980F819
:105310008C204A7908E00000100C002020100020AA
:105320008F070020100F002080F88D208A7980F8E8
:105330008E20C97980F88F106B490A7880F8902008
:105340004A7880F891208A7880F89220CA7880F88C
:1053500093200A7980F894204A7980F895208A79F8
:1053600080F89620C97980F897105F4908310A784B
:1053700080F898204A7880F899208A7880F89A20D6
:10538000CA7880F89B200A7980F89C204A7980F8B6
:105390009D208A7980F89E20C97980F89F10524913
:1053A00018310A7880F8A0204A7880F8A1208A78FD
:1053B00080F8A220CA7880F8A3200A7980F8A42077
:1053C0004A79C2F3400363F35F0280F8A5208A792B
:1053D00080F8A620C97980F8A710434920310A78BF
:1053E00002F0010280F8A8204A7880F8A9208A7883
:1053F00080F8AA20CA7880F8AB200A7980F8AC201F
:105400004A7980F8AD208A7980F8AE20C97980F891
:10541000AF10354928310A7880F8B0204A7880F8F2
:10542000B1208A7802F0030280F8B220CA7880F8AE
:10543000B3200A7980F8B4204A7980F8B5208A79B7
:1054400080F8B620C97980F8B710274930310A783A
:1054500080F8B8204A7880F8B9208A7880F8BA2095
:10546000CA7880F8BB200A7980F8BC204A7980F895
:10547000BD208A7980F8BE20C97980F8BF101A490A
:1054800038310A7880F8C0204A7880F8C1208A78BC
:1054900080F8C220CA7880F8C3200A7980F8C42036
:1054A0004A7980F8C5208A7980F8C620C97980F8C1
:1054B000C7100D4940310A7880F8C8204A7880F832
:1054C000C9208A7880F8CA20CA7880F8CB200A7967
:1054D00080F8CC204A7980F8CD208A7980F8CE20D7
:1054E000C97980F8CF1010BDCF0700207CB501210D
:1054F000082000F095FC4FF40050ADF80400102493
:105500008DF8074001208DF8060001A91548FEF727
:105510005FF90121092000F083FC01211248FEF708
:10552000A9F90820ADF8000004208DF803000F4E03
:1055300003258DF8025069463046FEF749F90821E7
:105540003046FEF7CAF9ADF800408DF803408DF8FB
:10555000025069463046FEF73BF910213046FEF70F
:10556000BCF97CBD0014014000023000000C014079
:10557000FEE7000038B50121082000F051FC4FF48F
:105580004060ADF8000048208DF8030003201B4D5B
:105590008DF8020069462846FEF71AF929152846B3
:1055A000FEF794F9164CE914607020702846FEF757
:1055B0008DF9E070A070FEF7B1F9A080E08011488D
:1055C00090F84A10104849B101290BD002290FD098
:1055D00003290CD1C17841F0030107E0C17821F023
:1055E000030103E0C17821F00301491CC17038BDFB
:1055F000C17821F00301891CF8E70000000C01408C
:1056000090080020A80200208F0700202DE9F0411B
:10561000444D4FF480612846FEF758F90446E914DA
:105620002846FEF753F9DFF800810746002598F871
:1056300000002E46844205D088F80040FEF76EF93F
:10564000A8F8040098F80100844209D0B8F80400D2
:10565000FEF74CF91E2803D388F80140A4B30025B7
:1056600098F802004446874203D0A770FEF756F927
:10567000E080E078874207D0E088FEF737F91E28FF
:1056800002D3E7701FB30026607828490028087904
:105690001FD020F002000871E278EAB120F001008A
:1056A00008710DB1002E2DD155EA06002AD0204BED
:1056B000DA7802F00300032800D90320002475B132
:1056C00003280CD2401C10E0FFE70125C8E70126A3
:1056D000DAE740F00200DEE740F00100E0E726B143
:1056E00018B1012810D0401EC0B260F30102114968
:1056F000DA7098B1012803D0022801D0032801D123
:1057000081F84A00BDE8F0810B4D6D6CB5F5FA6F7C
:10571000EBDA8978C906E8D50020E6E781F84A4047
:10572000F0E70000000C0140900800209F070020D7
:105730008F070020A802002038010020704700F0E9
:105740001F02012191404009800000F1E020C0F8D3
:105750008011704700F01F02012191404009800034
:1057600000F1E020C0F88011704700F01F02012115
:1057700091404009800000F1E020C0F8001170471E
:1057800000F01F02012191404009800000F1E0205B
:10579000C0F800117047000070B50F23C47801787D
:1057A0000122F4B1144C2468457804F4E064C4F593
:1057B000E064240AC4F10406E3408478B5401C4048
:1057C0002C4301F1E021230181F80034007800F03E
:1057D0001F018A404009800000F1E020C0F800214C
:1057E00070BD01F01F0082404809800000F1E020F8
:1057F000C0F8802170BD00000CED00E002490843B4
:1058000002490860704700000000FA050CED00E056
:105810002DE9F05F00261D20FFF791FF704CDFF8A7
:10582000C4B1A4F1B800A77E90F83810DFF8B8E151
:10583000DFF8B8A100258F427ED0E776A176626AB4
:10584000036B5A434FEA12499BF80820120702D50E
:105850001EF8012000E00A4694F812C0BCF1010FC6
:1058600009D004EB4206B6F902C0C4F828C0B6F964
:105870000460E6620CE043F6FF7CC4E90A5C90F841
:105880003DC05FEACC7C01D012B102E0052A00D114
:10589000012600EB47074FF0804CBF893F04B7FB60
:1058A000F3F3E361476BBCFBF7F7276294F813C08F
:1058B000BCF1000F06D0BCF1010F05D03B4403EB57
:1058C000D3735B10636201E03B466762DFF820C17F
:1058D0004FF6FF7707EA8307ACF808709AF8007074
:1058E00090F80A8090F83DC0082F08F003070CF0EC
:1058F000030C05D067450BD1B8F1000F05D008E0C7
:10590000674505D0B8F1000F03D05B42636200E049
:105910006562C6B1636A002B03D006DD228D05E007
:105920000AE0344B33F8122000E0A28DA4F8602086
:10593000227822F0200222709AF80020042A07D050
:10594000082A05D019E0B4F8603003EB0902EDE74E
:1059500080F8405065629BF80800000707D51EF8E4
:105960000100254901EB400030F8020C03E021481A
:1059700000EB41004088A4F860002049606A098873
:105980003E314843B4F8601001EB204006B21D20C0
:10599000FFF7EBFE606A002807D021784FEA8160AC
:1059A0000ADD002804DAA08D09E0B4F8600006E002
:1059B000E06AB04208DB0CE0002802DA208D208289
:1059C00008E0A06AB04204DD208241F0200020708F
:1059D00000E02682257565752586BDE8F09F0000EC
:1059E000F0010020A8020020DCBB00084F070020C7
:1059F000A40B0020EEBB000808BC000824040040F3
:105A000043184FF48042934210DD904202DD10466D
:105A100000210BE0914202DD0020114606E08003E8
:105A2000B0FBF3F000B2C0F5804109B241EA00409A
:105A30007047F0B541F2F1130022C3600E24826278
:105A400004824BF2660508264561068343F6FF771C
:105A50004283878340F2492E4FEA873CC0F808E032
:105A6000C0E9082CCB608A620C824D610E834A83A8
:105A70008F83B4208860C1E9082CF0BD00218162C9
:105A80000949C1600E210182084941610821018351
:105A90004FF44041418343F6FF718183090701625E
:105AA0000349416270470000B6A001001C0C0100D0
:105AB00000C0FF0F064941F6816008800548016873
:105AC000054A01F4E06111430160BFF34F8FFEE727
:105AD000442C01400CED00E00400FA05F8B501216A
:105AE0000D2000F09DF94FF4E060ADF8000018249F
:105AF0001D4E8DF8034003258DF80250694630464F
:105B0000FDF766FEB1153046FDF7E7FE711530462C
:105B1000FDF7E3FE31153046FDF7DFFE4FF4604040
:105B2000ADF800008DF80340104C8DF80250694626
:105B30002046FDF74DFE61142046FDF7D0FE4FF4E0
:105B400080412046FDF7CBFE4FF400412046FDF793
:105B5000C6FEA014ADF8000048208DF80300694689
:105B60002046FDF735FEF8BD00080140000C01405D
:105B70002DE9F0410121CE028CB0304600F050F901
:105B8000DFF87081404601F051FC08A801F07AFE70
:105B90004FF45860ADF824000024ADF820402020D8
:105BA000ADF822000125ADF826408DF8285008A94F
:105BB000404601F019FE0021404601F06CFE4FF610
:105BC000FF71404601F071FE01220021404601F0C4
:105BD000FDFD0121404601F0E5FB04A801F0FDFBBD
:105BE000ADF81060A802ADF81200ADF814408120A5
:105BF000ADF816002803ADF81800ADF81A40ADF85E
:105C00001C4004A9404601F0D7FBADF8084008202D
:105C1000ADF80A006027ADF80C408001ADF80070C7
:105C2000ADF80440ADF80E00ADF80240ADF8064006
:105C30006946404601F0BAFC6946404601F0FCFC6A
:105C40006946404601F042FDADF8045040F614505C
:105C5000ADF80070ADF80600ADF80840ADF80C40A6
:105C6000ADF80250ADF80A40ADF80E406946404626
:105C700001F070FD0121404601F0B8FB08214046CB
:105C800001F0D4FC3146404601F016FD08214046A3
:105C900001F05AFD3146404601F08EFD702140462C
:105CA00001F097FD18208DF82C008DF82D408DF80F
:105CB0002E408DF82F500BA8FFF76EFD0D480C30CD
:105CC000018841F0800101800A481430018841F0C8
:105CD00001010180001F04800121404601F090FB7A
:105CE0008DF828500121404601F094FB0CB0BDE82E
:105CF000F0810000002C0140704740F213414160E8
:105D0000082181608621C1604FF4804101614942D0
:105D1000416100210162C162704701627047000069
:105D200010B501884288891A09B20183B1F5005F74
:105D300002DBA1F5804104E011F5005F02DC01F512
:105D400080410183B0F9182041685143C1618368E3
:105D5000846A5343C2681B12624303EB2222036A24
:105D60001A44114402628A13426241698A4203DB87
:105D700001698A4200DC11468A1AC0E90A21028EB2
:105D80004FF40373594302EBA13202860B4A127897
:105D9000082A04D10A4A936F03EBA1319167B0F945
:105DA0003010B1F5804F02DDA1F5804103E00029FC
:105DB00002DA01F58041018610BD00004F07002086
:105DC000240C0020034A516821F4404101435160F2
:105DD0007047000000100240044A0029516901D0B8
:105DE000014300E081435161704700000010024010
:105DF000044A0029D16901D0014300E08143D16107
:105E00007047000000100240044A0029116901D0C7
:105E1000014300E08143116170470000001002401F
:105E2000044A0029916901D0014300E08143916156
:105E30007047000000100240044A0029D16801D0D8
:105E4000014300E08143D160704700000010024030
:105E50002DE9F041274C4FF4807631462046FDF77E
:105E600035FD850080212046FDF730FD45EA4005DF
:105E700040212046FDF72AFD0543EDB2314620467C
:105E8000FDF724FD870080212046FDF71FFD47EA2E
:105E9000400740212046FDF719FD0743F8B2A8420C
:105EA000DBD131462046FDF711FD870080212046D9
:105EB000FDF70CFD47EA400740212046FDF706FDAF
:105EC0000743F8B2A842C8D131462046FDF7FEFC90
:105ED000870080212046FDF7F9FC47EA4007402172
:105EE0002046FDF7F3FC0743F8B2A842B5D1284697
:105EF000BDE8F0810010014010B50268416802FB66
:105F000002F301FB0133B3F1805F11D91B0E103B8B
:105F10000A4C9BB212B234F8133009B25A435943B7
:105F200042F38F3241F38F31C0E90221012102E0B7
:105F3000C0E902210021017410BD0000C8B10008B1
:105F40002DE9F05FFE48FF4902880B889A1A92B249
:105F50000F2A74D309880180FB480024827852B14B
:105F6000818AB1F5967F02D2491C818204E0848245
:105F7000521E827000E084828246C078401E012852
:105F80000ED8BAF8161047F230525046914203D25A
:105F9000491CAAF8161005E0C4828AF8034001E003
:105FA000AAF81640E94802468189D2884B0703D4F3
:105FB0008B0701D4CB0702D042F4007201E022F437
:105FC0000072C280080702D4E048C90604D5DF4841
:105FD000C18841F0010102E0C18821F00101C180C6
:105FE000DA48FDF71BFADA48B0F93A00B0F5804F0D
:105FF00002DAD749401C02E0D5494FF48040DFF86F
:1060000054B34887DFF84093DBF8503041F6CC407A
:1060100009F13809834205DDD9F8081021F0100193
:10602000C9F80810CC49DFF83483CD4E0A88CD4832
:1060300032B1521E0A8089F80F4034700BE027E11C
:106040009AF8021009B1032916D998F8002022F015
:10605000020288F80020B9F84210D9B3494631F855
:10606000422F521E0A8098F8005025F0020588F849
:10607000005089F80F403FE0B9F8421059B3B34AD5
:10608000D1884F041CD49289D70619D4170717D486
:106090000F0615D48F0613D40F0511D44F0603D560
:1060A000B14F3F783F060BD54F0709D4CF0507D432
:1060B0000F0705D48F0403D4C90601D4D107CDD06E
:1060C000AA4989F80F40AA4A3470CC83148081F819
:1060D0002840C3E704E0FFE7A64A49F68161118042
:1060E00098F8002042F0020288F800203178012957
:1060F00003D10178062900D134703178DFF878E2D5
:106100009E4D01270A296ED2DFE801F0F9C205C2CF
:10611000F8F7C26DF6F502F0FFF9BAF8221040F672
:106120002820491C8AB2AAF82220DBF844108142B8
:1061300002DAAAF8224013E0854840F6CC43C06852
:1061400098420DDBB8F9040043F69913984207DB37
:10615000B2F5FA7F04D32A7812B9AAF822402F7038
:10616000874A108868B19AF806305B1CDBB28AF85F
:106170000630022B05D383488AF8064003885B1C4F
:10618000038099F80F00C846092812D002287CD055
:10619000A8F83441B8F84400A146D0B141F288349F
:1061A0004846AAF82290A14222DA297801291BD078
:1061B0001EE063484430FDF7DBFCFDF7A5F9DBF892
:1061C0004410CAF8341041F27C510920CAF8241056
:1061D000C0E2A88AA8F83400E86A6863A86A28635D
:1061E000A8F844703AE0C7E166492870088010803A
:1061F00098F84A10022908D06349C978B7EB511FB3
:1062000010D098F82C1151B104E098F82C1109B96C
:106210006FF0A200C8F8DC0088F8EE7008E06FF4B8
:106220000560F7E7C8F8DC0088F8EE00CAF82C0033
:106230005548B8F93410C078B7EB501F06D0B8F8FD
:10624000DC00642300B240F2DC5203E04FF47A73C6
:106250005A00002000F0BAFBA8F834004A484B4925
:106260004FF49A73C078B7EB501FDBF8440011D09D
:10627000B0F5FA7F0CDAB5F90A00984208DC00BFE5
:1062800086F8009088F8EE9000E01EE0A1F81A90E1
:10629000BDE8F09F40F2DC52904203DAB5F90A20E3
:1062A0009A42EDDDB8F8442040F6C413521C92B275
:1062B000A8F844209A42E3D2254AD268002AE7DCB3
:1062C00042F6E0629042DBDAE2E7B8F8342140F6C9
:1062D000B830824207D21A4B183B1B78DB0702D139
:1062E000521CA8F8342193B240F2DC52934207D8F2
:1062F00042F6CC4008E0D2E0ACE0F9E0F4E0FCE0AB
:10630000A8F8340143F26660E867CAF834108AF8E6
:106310000B701F4EA8F8444088F8EE40707F554639
:10632000C0B3F07FB8B3B8F82C00B8F9341000B29D
:106330000A23052200F04AFBA8F83400F4772BE08A
:10634000D80A00205807002070020020100C0020FE
:1063500040050020380100205C070020F2050020E5
:106360004F0700205007002020070020400A00208F
:1063700006000020442C0140580200204C00002060
:10638000080000200A000020B70700204C0B002066
:10639000300E002012E044E086F81D40B8F91A01E2
:1063A000B8F91811884240DAE97901F1010111F0D8
:1063B000FF01E97140D0EC71401C38E04FF480409F
:1063C000A8F8E800D8F82C10814200DA0846F54910
:1063D00000B2288491F84D1051B998F84A1039B19B
:1063E000B8F80820C2F3C003C2F30022934204D1DC
:1063F0003623B8F93410052209E0012903D0022917
:1064000001D0032906D0B8F93410DA23242200F091
:10641000DDFA07E0B8F9341040F2991340F26662F1
:10642000F5E7A320A8F83400B8E703DD801EA8F83C
:106430001A0101E0A8F81A11B8F934004FF48041AC
:10644000884202DDA8F8341022E70028FCDAA8F818
:1064500034401DE7D9F8E0204EF6602148468A42D4
:1064600002D2521CC0F8E020C27B082A03D1D0F827
:10647000E0208A420FD33470816821F4006181608A
:10648000CA0502D521F0080101E041F00801816050
:10649000C9F8E040FCE6BDE8F05F02F0C7BF99F83C
:1064A0000F004F46092803D0BC8689F80F4053E1FE
:1064B000DAF828005546401CCAF82800022809DDF1
:1064C000A88E012301B2A88C052200B200F07EFA4A
:1064D000AC626863B448A98E0180BBF84410418067
:1064E000FDF75EFBB886D3E6BDE8F05F04F010BDB3
:1064F0009EF8000009287DD0CAE689F8114199F874
:106500002C2162B143F31101C9F8DC40A74A8B0387
:10651000E962891093628A03A962A5498A62AAF88E
:106520002240DBF8442041F288318A4207DA297898
:10653000012904D19F492C700C809F490C809F4AEF
:10654000DFF87CC21188491C8BB29E491380C82B8E
:1065500004D391F80080B8F1010F1AD0B3F57A7F17
:1065600004D391F80080B8F1020F12D0B3F5FA6F9E
:1065700002D30B78032B0CD099F80F10891E082931
:106580007ED2DFE801F010ABEBFD057D850410E65F
:106590007EE60C708C491480CA8822F40062CA809E
:1065A0008CF80070E8E7DBF84410D846822904DA5A
:1065B0000178062901D00470E5E0FDF7DFF998F8CD
:1065C0000000400613D58148807804280FD0D8F801
:1065D0004410404682290ADA817A98F83D0001F099
:1065E000030100F00300814201D001F045FEB346F3
:1065F000307800E0B0E00628CAD088F83F40D8F8EC
:1066000050006A4940F311008203E86280108A62F8
:106610008103A862664846468162FCF775FF8AF8E6
:106620000B70B9F81801A9F81A01706C4D46B0F555
:10663000437FA9F8864010DD4FF48040A5F8840020
:10664000A86840F48060A86096F8381005299FD1AA
:1066500040F01000C9F8080016E04FF48041A5F89A
:106660008410A96821F48061A96040F28A218842DF
:1066700004DA3078400601D402F0BAFDA86800E0E0
:1066800088E040F01000A86002208BF80000FFE5D1
:10669000DBF84410B1F5437F02DA017806298AD18C
:1066A0004B48017821F040010170FCF72DFF43F6C3
:1066B000FE70A9F81A0109F1E005FDF75FF94548F8
:1066C00010F8341F21F00101017039492C608C62EF
:1066D00036498C62082131704464D9E53A488079A2
:1066E000C006D4D4DBF844005D46B0F57A7F33DDD4
:1066F000FDF744F92878400611D5344880780428FD
:106700000DD0686C82280ADAA87A95F83D1000F05E
:10671000030001F00301884201D001F0ADFD85F8CE
:106720003F40B5F85000A9F8340001B24FF4804062
:106730004C46814200DDA086FCF7E6FEA06840F4EE
:106740008060A06095F838100529A0D140F01000B5
:10675000A060022030709BE5347099E5DBF84410AE
:10676000B1F5437F02DA0178062998D11648C1882D
:1067700021F02001C180FDF701F90420EAE7FFE7DD
:106780000078062801D0377082E509208EF80000D5
:106790000520DFE70D498C70047085F85E40A9F88C
:1067A000344075E5680E00201C0B0020100A002004
:1067B000E00900200A00002008000020100100204D
:1067C0000E01002012010020100C00205C040020AB
:1067D0005E070020240C002030B585B00121042084
:1067E000FFF71EFB4FF40040ADF8100048208DF875
:1067F000130004A91848FCF7EBFF01210846FFF736
:10680000F7FA40F68C20ADF8040003240020ADF820
:106810000040ADF80200ADF806004FF08045694633
:10682000284600F0E1FF1C208DF80C008DF80D408B
:106830008DF80E4001208DF80F0003A8FEF7ACFF85
:1068400001221146284600F0A9FE0121284600F049
:10685000D7FD05B030BD00000008014070470000C2
:106860002DE9F041304CE07800285AD120780028FA
:1068700057D0401E10F0FF00207052D14FF4967098
:10688000208272B6294F45F2AA50A7F87200002064
:10689000FCF718FE264D13202860FCF725FEA8BB48
:1068A0003420E86002202861224E6E61286940F0A1
:1068B00040002861FCF718FE40BB00211E4A084634
:1068C0005FEA255312F800C0BCF1FF0F00D0012190
:1068D000401C80B29842F5D3C1B9C4E90676392686
:1068E0000127A06910F8011B10F8012BA061E069D5
:1068F00001EB022102886A612F6120F8021BE0612E
:10690000FCF7F2FD10B9761EB6B2EAD20120FCF710
:10691000D9FD62B601F004FD0848816821F4804188
:106920008160BDE8F08100004C070020680E002067
:106930000020024000FC000800FC0008A802002023
:106940001948016841F010010160016821F003015C
:106950000160016841F00201016014484168416032
:1069600041684160416841F480614160416821F4BF
:106970007C11416041680E4A11434160016841F059
:106980008071016001688901FCD5416821F0030133
:106990004160416841F0020141604168C1F38101F9
:1069A0000229FAD170470000002002400010024086
:1069B0000000280830B5044C039D6080A180E2806F
:1069C0002381658130BD0000040C00200A4482420E
:1069D00001DA10B27047C91A8142FBDD08B2704774
:1069E0002DE9F04F4A48DFF82CA1DFF82CB1C17F28
:1069F000477A046849480022DFF82C91466C4848E1
:106A00004FF0010E802985784648836834D301F021
:106A10001F0C5AF82C100C420146096802D041F4B0
:106A2000805101E021F4805101605FEAC14C1ED425
:106A30005FEA814C1BD599F80AC0C8465FEACC7C56
:106A40000BD05FEAC31C12D4A8F80A209BF8008080
:106A500028F002088BF8008009E0322E07DC5FEA9C
:106A6000857C04D55FEA035C01D4A8F80AE04FEA0C
:106A7000113C6CF34D310160802F24D307F01F07C8
:106A80005AF827100C42016802D041F0040101E0DD
:106A900021F0040101604C0711D44C050FD599F881
:106AA0000A70FF070BD0DF0109D4A9F80A209BF870
:106AB000007027F002078BF80070C0F89C208C084B
:106AC00064F38A21016099F80A40E40719D1174C50
:106AD00094F86440012C14D1322E10DC046866074F
:106AE0000DD51B050BD4E30409D5AB0707D5D0F8AA
:106AF0009C304EF66024A34205D9A9F80AE0C0F8FC
:106B00009C20BDE8F08F5B1CC0F89C30F9E70000CA
:106B1000F805002018B70008F20500203801002011
:106B20009F070020A8020020100C0020680E002003
:106B300010B5FAF75FF90F48018821F002010180D2
:106B40000C49183109880C4A928E1144094A343292
:106B5000118008490C390A8842F001020A80011D9F
:106B60000A884FF6ED531A400A80018841F012015D
:106B7000018010BD0C0400405C040020130A037067
:106B80000A70704705484FF6FF620188491C89B2B8
:106B90000180914201D300210180704798080020B4
:106BA0000F4810B5016841F00101016041680D4ACC
:106BB0001140416001680C4A11400160016821F4F4
:106BC00080210160416821F4FE0141604FF41F0102
:106BD0008160FFF7B5FE05494FF00060086010BD09
:106BE000001002400000FFF8FFFFF6FE08ED00E095
:106BF0004FF0E02005494161054AF02182F8141D5B
:106C0000002181610721016170470000DFA50100BB
:106C10000FE000E02DE9F047DFF8B090B9F8000090
:106C20004FF0000400064DD5294D6888401C68804F
:106C3000FBF730FC274E284B284832786A7093F8CF
:106C40000080072726494FF0C80CB8F1010F03D088
:106C5000244AD288E2B12EE072B1012A12D0C28851
:106C600042F40062C280886840F00400886003201B
:106C70002870052030701BE0828942F00802828172
:106C80000120F5E7828942F0100282810220EFE7BD
:106C9000154A15786D1CEDB21570032D08D91470C6
:106CA000C28842F40062C280886840F004008860B4
:106CB0001F70A1F842C000204FF49661401C80B2C2
:106CC0008842FBD3A9F80040BDE8F087102C0140B2
:106CD0003C070020500700204F070020100C002028
:106CE000A8020020D80A002072020020704700008D
:106CF0002DE9F0434FF08040018A21F0010101822B
:106D0000AA48007800287CD1A94FF87B002878D1C8
:106D1000A848406C322874DCA7488068DFF89C9251
:106D20004104A74DB9F804004FF0000403D4401CFF
:106D3000A9F8040024E1002874D02978012611B1B3
:106D4000012912D013E14946B0F5BE7FFAD92E7061
:106D5000CC718C71EC702C72287A0A18401CC0B26D
:106D6000147228720F28F7D301E1B9F802204946BE
:106D7000824201D9EE7100E0EC7190488A790830C6
:106D80000F2A15D2CB79082B0BD2C3F10708EB7968
:106D900012F800C003FA08F363441354CA79521C72
:106DA000CA71CA79082A03D18A79521C8A71CC71B6
:106DB00099F80610C8460F2973D10D21FBF702F987
:106DC000A881010A6970C0B2A87088F8064098F8D6
:106DD00016208A4265D198F81510814261D198F841
:106DE0000BC07849032302227748BCF1000F10D072
:106DF000BCF1010F02D0BCF1020F14D080F86A2060
:106E000000E0C7E091F800C02CF00C0C0CF1080C6D
:106E10000FE080F86A6091F800C02CF00C0C0CF1C7
:106E2000040C06E0A5E080F86A3091F800C04CF050
:106E30000C0C81F800C098F80C10B6EB111F04D1AF
:106E400080F86E4087F84A400EE0B2EB111F04D183
:106E500080F86E6087F84A6006E0B3EB111F03D13B
:106E600080F86E2087F84A200B0717D001F00F0139
:106E7000012901D0022915D080F86C602C7198F896
:106E80000D102A7906FA02F30B406B71082A41D2E1
:106E9000DFE802F00B0F4016212C333A80F86C40EB
:106EA000ECE764E080F86C20E8E713B380F870400A
:106EB00030E013B180F850602CE080F8504029E0B9
:106EC00023B180F8656087F8076123E080F86540AA
:106ED00087F807411EE023B187F8F94080F84D405C
:106EE00018E087F8F96080F84D6013E013B180F87E
:106EF00068600FE080F868400CE013B180F86660CD
:106F000008E080F8664005E013B180F8676001E0B2
:106F100080F86740521CD2B22A71082AB1D398F87F
:106F20000E108A0704D587F8F56080F8646005E0E4
:106F3000264A87F8F54080F864405481C90702D09A
:106F400080F8294001E080F8296098F8111000F8D5
:106F50006D1FC2781E48012A1ED001B3012921D01D
:106F60004FF48051A0F876101A493C200870A9F817
:106F70000240A9F80440B9F80210491CA9F802100F
:106F8000B9F80210B1F5FA7F04D940F2F511A9F869
:106F900002102C70BDE8F08344F21C71E2E74FF45C
:106FA0000051DFE741F25551DCE700004F070020B8
:106FB000A80200203801002000100140500E0020DF
:106FC000D8060020D4040020680E0020100C0020F9
:106FD000400500204C0700202DE9F05FFCF7CEFCB7
:106FE0008E4D2888A5F10406C0070AD0308820F00D
:106FF00008003080288820F00900288002F0F8F886
:10700000D9E02888DFF81892DFF81882864C8007CC
:107010001AD5B9F8001041F00101A9F80010B8F82C
:107020000000804914315030088028884FF6F9510B
:1070300008402880308840F004003080FEF708FFC8
:1070400084F83C00BDE8F09F2888784F40072888E6
:1070500071D520F004002880FEF7FAFE94F83C1069
:107060008142EFD1308820F004003080FCF7A6FE8A
:107070002078410605D594F8541094F83B209142AD
:10708000E0D03978400621F00201397004D5FDF7CF
:107090001FFE97F82F7004E094F83C00FCF7C0FC4A
:1070A0000746DFF880B140F68C2A0BF1180B062F4B
:1070B00047D294F83800B8423ED03846FCF734FC4A
:1070C0002078C00716D094F83A0094F8391000F0F0
:1070D0000302914206D0A17A00F0010001F0010103
:1070E000884215D1FCF7D2FDF9F7D0FEFCF7FEFE81
:1070F000384689E0FCF7CAFDF9F7C8FEFCF7F6FE52
:107100003846FCF7E3FD207840F00100207099E755
:10711000288820F008002880206B810801EBD0002F
:10712000504515D2B8F800100844ABF8000030887C
:1071300040F0080003E00DE0308820F008003080C7
:1071400080E7B9F8001041F00101A9F80010DFE76D
:107150005046E7E70007288831D520F0080028804E
:10716000308820F008003080FEF772FE84F83C0082
:10717000FCF724FE387820F00200387020784006B2
:1071800004D5FDF7A5FD97F82F5004E094F83C00D6
:10719000FCF746FC0546062D08D294F83800A842B4
:1071A000B5D0FCF773FDF9F771FE2AE02048C188DD
:1071B00041F04001C180BDE8F05FFCF775BEC0063C
:1071C000288825D520F010002880308820F0100075
:1071D000308097F838000C2802D2401C87F838001D
:1071E000387840F002003870FDF772FD97F82F50A4
:1071F000787884F8390094F83800A84287D0FCF7F2
:1072000045FDFCF773FE2846BDE8F05FFCF75EBD68
:107210004EF2BE110840288014E700001004004020
:107220000004004024040040380100205C040020D9
:10723000100C00202DE9F04F514F85B0388820F018
:10724000010038804E480026103006804D4CDFF893
:1072500038A14FF0010894F85C0042F63029C107CC
:1072600074D072B64948816941F4007181618169C5
:1072700041F4806181614FF40040FEF7A3FD444D6D
:1072800000212846F9F74EFB00212846F9F740FB7C
:10729000DFF800B100215846F9F73AFB00213E48DB
:1072A000FBF7CEFB2846F9F75FFC5846F9F75CFC84
:1072B0004FF46020CDE902068DF8056000968DF848
:1072C00010808DF8048069462846F9F7DFFC012319
:1072D0001A460F212846F9F72AFD01212846F9F719
:1072E00017FB00204946401C80B28842FBD3284649
:1072F0002E600121F9F75AFD28688007FCD5244843
:107300004C30006894F85C1021F001012144A1F890
:107310005000F9F711FB62B6FDF7E8FB47F6906104
:10732000AAF8001094F85C00401CC0B284F85C001D
:107330000C2822D212491431A1F80080388840F07C
:107340000100388005B0BDE8F08FFFE7134920F059
:107350000100085A12490880114945F658000839B9
:1073600008800F4846F65801001F01800C49202074
:107370000C390880AAF80090D4E70320A070E1E758
:10738000000800405C0400202C080040001002406F
:10739000002401400028014008000240D4B2000847
:1073A000202C01400029018802D041F0800101E039
:1073B00021F080010180704710B50A884B88CC8885
:1073C0001A438B8823431A430B891A434B898989B3
:1073D0001A430A43A0F8442010BD002101804180D7
:1073E0008180C1800181418181817047002981882C
:1073F00002D041F0010101E021F0010181807047DC
:107400000029018802D041F0010101E021F00101D1
:1074100001807047002930F8441F02D041F4004138
:1074200001E0C1F30E010180704700004B4910B527
:10743000884202D10121C41486E0B0F1804F09D006
:10744000474988420DD101210220FEF7DDFC0021D1
:10745000022064E001210846FEF7D6FC002101204D
:107460005DE04049884206D101210420FEF7CCFCB2
:107470000021042053E03C49884206D10121082024
:10748000FEF7C2FC0021082049E03849884206D1B5
:1074900001211020FEF7B8FC002110203FE0344904
:1074A000884206D101212020FEF7AEFC00212020D9
:1074B00035E03049884202D10121441444E02E498C
:1074C000884202D10121CC043EE02C49884202D1FD
:1074D00001210C0538E02A49884202D101214C05DE
:1074E00032E02849884206D101214020FEF78CFC79
:1074F0000021402013E02449884206D10121802048
:10750000FEF782FC0021802009E0204988420AD150
:10751000841501212046FEF777FC00212046BDE8B6
:107520001040FEF771BC1A49884202D101210C04B7
:107530000AE01849884202D101214C0404E01649AE
:1075400088420AD101218C042046FEF775FC2046B2
:10755000BDE810400021FEF76FBC10BD002C0140BB
:107560000004004000080040000C004000100040F3
:107570000014004000340140004C01400050014024
:107580000054014000180040001C00400020004052
:10759000004001400044014000480140002A828927
:1075A00001D00A4300E08A438281704730B5028CE3
:1075B00022F001020284028C8388048B22F00202F2
:1075C00024F073050C882C430D8915434A882A43FF
:1075D000114DA8420BD0114DA84208D0104DA84221
:1075E00005D0104DA84202D00F4DA8420DD122F077
:1075F00008054A8923F440732A4322F004058A8847
:107600002A438D891D43CB892B4383800483C988FA
:107610008186028430BD0000002C0140003401400E
:10762000004001400044014000480140028B22F02C
:1076300008020A430283704770B5028C22F01002E0
:107640000284028C8488038B0D8823F4E6464FF66F
:10765000FF7303EA052535430E8922F0200203EA71
:10766000061616434A8803EA02123243104EB0420D
:1076700002D0104EB04215D122F080064A8924F47F
:10768000406403EA0212324322F040068A8803EA89
:10769000021232438E8903EA86062643CC8903EA26
:1076A0008404344384800583C9880187028470BDC3
:1076B000002C014000340140028B4FF6FF7322F48E
:1076C000006203EA012111430183704770B5028C07
:1076D00022F480720284028C8488838B0D8823F0CC
:1076E00073031D4322F400730E894FF6FF7202EA02
:1076F00006261E434B8802EA03233343104EB04252
:1077000002D0104EB04215D123F400664B8924F408
:10771000405402EA0323334323F480668B8802EA51
:10772000032333438E8902EA06162643CC8902EAF4
:107730000414344384808583C9888187038470BDA1
:10774000002C014000340140828B22F008020A43E1
:107750008283704770B5028C22F480520284048CBC
:107760008288838B0D8823F4E6464FF6FF7303EA85
:107770000525354324F400560C8903EA04343443C8
:107780004E8803EA06362643094CA04202D0094C33
:10779000A04205D122F480448A8903EA821222435E
:1077A00082808583C988A0F84010068470BD0000DF
:1077B000002C014000340140828B4FF6FF7322F40D
:1077C000006203EA012111438183704701858282AF
:1077D0007047828822F07002828082880A43828009
:1077E0007047A0F84010704730B502881B4B1C4C06
:1077F00098420DD0A0420BD0B0F1804F08D0194D67
:10780000A84205D0184DA84202D0184DA84203D175
:1078100022F070054A882A43154DA84206D0154D1E
:10782000A84203D022F44075CA882A4302808A887D
:1078300082850A88028598420AD0A04208D00E4A62
:10784000904205D00D4A904202D00D4A904201D19B
:10785000097A01860121818230BD0000002C01409F
:10786000003401400004004000080040000C0040CB
:10787000001000400014004000400140004401405E
:10788000004801404FF6FF71818000210180C180D6
:107890004180017270470029018802D041F0020145
:1078A00001E021F00201018070470029018802D027
:1078B00041F0040101E021F0040101807047000063
:1078C000194810B54079002300F003011748022938
:1078D00027D0174A01881488611A89B201240F2918
:1078E0000BD3118801808168002900DA49420129FF
:1078F00003DD10490978022905D0417F012906D00E
:107900001188418010BD4477C37711884180418838
:107910001288511A89B240F21A629142F2D3C477A6
:1079200010BD437710BD0000B7070020300E0020C7
:10793000580700204F07002080092830FF2801D970
:10794000FF207047C0B270472DE9F041B1F90250F5
:1079500000231E240F22854203DDB1F90000BDE89B
:10796000F081B1F97A50854202DAB1F97800F6E790
:1079700001EB8205B5F90250854201DA134600E0B9
:107980001446E21852085D1CAA42F1D101EB8203B1
:10799000B3F90240844206DAB3F9067031F9225095
:1079A000B3F9046005E033F9027C31F9225033F970
:1079B000046C001BC11789013A1B41EA9061D3177F
:1079C0008001F8F7AFFB721BA0FB024601FB0261CE
:1079D000D31700FB0310810641EA9410284400B23B
:1079E000BDE700002DE9F04FDFF8B8B16A48DFF8D5
:1079F000AC91DFF8ACA190F80EC0BBF91A70BBF9DE
:107A00001C60BBF91850BBF96C10BCF1070F48D2D1
:107A1000DFE80CF08D041A30485E7600D9F80020BB
:107A2000C284DAF800200285C28C038DA7EB8202A3
:107A300012B2A6EB83034A431BB2594342F3CF224F
:107A400041F3CF23D11870E0D9F800208284DAF80E
:107A500000200285828CA5EB820213B2028D4B437B
:107A6000A6EB820212B243F3CF24514341F3CF235A
:107A7000E11814E0D9F800200285DAF800208284A9
:107A8000028D838CA6EB820212B2A5EB83031CB29B
:107A90004A43614342F3CF2341F3CF2419194942AA
:107AA0000AB244E0D9F80020C284DAF800208284C7
:107AB000C28C838CA7EB820212B2A5EB83034A43EC
:107AC0001BB2594342F3CF2241F3CF24111914E0E2
:107AD000D9F800208284DAF80020C284828CC38C1A
:107AE000A5EB820212B2A7EB83034A431BB242F317
:107AF000CF24594341F3CF22A11849420BB216E0DB
:107B0000D9F800200285DAF80020C284028DC38CE7
:107B1000A6EB820212B2A7EB83031CB24A4342F3E4
:107B2000CF23614341F3CF22991849420CB2BBF9EC
:107B30001E50594605F21E56A64201DACE8306E0D3
:107B4000A5F21E55A54201DDCD8300E0CC83B1F93D
:107B5000204004F21E55954201DA0D8406E0A4F29D
:107B60001E54944201DD0C8400E00A84B1F9222005
:107B700002F21E549C4202DAABF8224008E0A2F264
:107B80001E529A4202DDABF8222001E0ABF822300F
:107B9000417B8173BDE8F08FA80200203C240140A6
:107BA0003C280140400500202DE9F047044670487C
:107BB000714E002702786F48022AB0F9341004D0C1
:107BC000082A6ED0092A6DD0CDE0C27B022A02D1EC
:107BD000B0F844205AB1A4F8421071810423B6F9D8
:107BE00008101A460020FEF7F1FE3081BBE0634921
:107BF000DFF88C81496A0D14E58090F84A1099B13C
:107C00000089DFF88091C0F3C001C0F300208142F9
:107C100023D1D8F8440040F2BA41884240DD40F612
:107C20006A1188420ADC15E0B4F9020040F2DA2158
:107C3000884279DD40F26A41884204DD0823B4F9C4
:107C400042101A464EE0A0F2DA20F8F7F4FB0022C8
:107C50004D4B56E0A0F2BA404FE04C480078C006C9
:107C60000CD5D8F8440041F2243188425CDD41F261
:107C7000D4718842E2DC00F6DC4020E04448DFF8C2
:107C8000149190F8701001290DD090F86F00012820
:107C900009D041480178C90746D04049098889B1CF
:107CA00042E05AE05DE0B4F9020041F6DC6188424E
:107CB0003ADD42F23411884210DC00F59270A0F5F2
:107CC00000501AE0B0F91000B4F90210A0F5967255
:107CD000914229DD00F5967291420BDDB4F9421014
:107CE00020231A460020FEF771FEA4F84200002867
:107CF00017DB1BE0081A00F59670F8F79CFB0022D2
:107D00004B46F8F704FB0E22F8F770FBF8F7CAFBB6
:107D100000B2C0F5804068438013A4F84200002DF3
:107D200004DCA4F8427001E0A4F842501C48B0F909
:107D30001210D8F85000081A718B01EB600000B2E5
:107D4000F082002800DCF782B4F94200B6F9161080
:107D5000884200DB0846708104E01248B0F87C00DD
:107D6000F9E77181378184F84070BDE8F087000041
:107D70004F070020A80200204C00002040050020F2
:107D80003801002000C09240000079402007002008
:107D9000680E002000C08240C00A002008000020B9
:107DA000D80A0020240C00202DE9F041B1F902503E
:107DB00000232B241522854203DAB1F90000BDE827
:107DC000F081B1F9AE50854202DDB1F9AC00F6E7C1
:107DD00001EB8205B5F90250854201DD134600E052
:107DE0001446E21852085D1CAA42F1D101EB82054B
:107DF000B5F90230834206DA35F9026C35F9044CE4
:107E000031F9221006E01E4631F92240B5F906305C
:107E1000B5F90410801B091BC5178911AD0345EA8C
:107E200090458703A1FB070CCA1702FB07C201FBA1
:107E300005219A1BD317F8F775F9000A40EA01608B
:107E4000001900B2B0F5804FB9DB43F6FF70B6E71A
:107E500070B5134C40F224452946204600F02CF81A
:107E600000281BD0204600F046F82946204600F0A6
:107E70001DF80C4C00212046FAF7E2FD2046FAF7E7
:107E80005DFEC0F164000849C0B20428087201D93F
:107E900000F0AEF9BDE87040FAF78EBE70BD00008C
:107EA0000038014058000240840600200A0A0121DF
:107EB0009140C9430180704730B501F01F02012491
:107EC0000025C1F3421304FA02F2012B0FD0022B5A
:107ED0000FD0838A4FEA11210088134204FA01F47B
:107EE00000EA040001D000B10125284630BD838995
:107EF000F0E7038AEEE78088C0F3080070470000CF
:107F000070B5214C2068214D400103D520492846F9
:107F1000F9F706F92068000104D51D492846FF310C
:107F2000F9F7FEF82068C00003D51A492846F9F78A
:107F3000F7F81948194A0178CB0712D192F82F3077
:107F4000012B0ED0FAF70CF82068C0F382611448B8
:107F5000072916D0216811F0E05F01D15521017089
:107F600070BD012382F82F3021F0010101700D480E
:107F700001680D4A01F4E06111430160BFF34F8FC6
:107F8000FEE70021EBE700000864004000640040C9
:107F900001000038000001384E080020DC0E0020EF
:107FA000580800200CED00E00400FA05F0B585B09B
:107FB000042000258DF808000702844C00950195E7
:107FC0008DF80A508DF8135039462046F9F708FA13
:107FD00001281DD17E4E06F8305FF9F71FF82068A2
:107FE00040F40040206079481430016821F001011C
:107FF0000160784D286800F0FBFD002176A001F0BB
:108000005BFE286039462046F9F7A2F8012030705F
:1080100002212046F9F7E4F901287CD16A460021C3
:108020002046F9F7B3FA01986E4920F06040886065
:108030009DF80A1008291BD16B4908440C2817D257
:10804000DFE800F0060BBDBDBDBDBD1752717CA3BE
:1080500064489DF80B106F309BE0624A002069462F
:1080600017320B18DB7A1354401CC0B20828F8D31F
:10807000A5E05C499DF80B004F3103090A7860F3D5
:10808000030263F30412430963F34512800960F3AA
:1080900087120A709DF80C0048709DF80D008870DA
:1080A0009DF80E00C8709DF80F000A7960F3000279
:1080B000400860F347020A719DF8100048719DF86E
:1080C00011208879930862F3010063F38300120999
:1080D00062F3071088719DF81220C87962F30600D8
:1080E000D20962F3C7104EE040489DF80B100170B2
:1080F0009DF80C1041709DF80D1001F00302827084
:10810000C1709DF80E1001719DF80F1041719DF81E
:108110001010817100E056E09DF81110C1719DF8BA
:10812000121001724BE02F489DF80B205730017858
:1081300062F30101920862F387012AE029499DF860
:108140000B205F31087862F30300120962F3071015
:1081500008709DF80C0048709DF80D20887862F337
:108160000600D20962F3C71088709DF80E00C8702F
:108170009DF80F0008719DF8100048719DF81100DE
:1081800088719DF81200C87119E016489DF80B100F
:10819000673001709DF80C1041709DF80D108170D2
:1081A0009DF80E10C1709DF80F1001719DF8101010
:1081B00041719DF8111081719DF81210C171022159
:1081C0002046F8F7C5FF05B0F0BD00000064004090
:1081D000DC0E00205C0800206465765F63616E3110
:1081E0000000000070070020FFFE00E720100020C4
:1081F00070B51D4D00242878432834D1687846286E
:1082000031D1A878502807D0512805D0812803D033
:10821000892801D0212826D1144E7071E978717215
:10822000A81C891CF9F706FFB072717A29440979F4
:108230003182884217D106F10E00017841F0020127
:1082400001700B48016841F020010160317A094852
:10825000002204E02B5D03552A55641CE4B28C42D5
:10826000F8D38078707170BD00090020840600206A
:108270000C0C0140A20D002070B51D20FDF76AFA1C
:10828000FCF726FD1D20FDF77BFA154890F82F100E
:10829000144D0623144C85F8381090F83B1095F8CF
:1082A0003B201143012A04D0022A07D0042A0AD015
:1082B00010E0827A8A420DD0007B09E0027D8A427A
:1082C00008D0807D04E0827F8A4203D090F82000AD
:1082D000884200D12370002085F8400070BD000066
:1082E0005C040020380100204F0700200B480021CB
:1082F0004180A0F1B8018A898280CB891A44C2806A
:108300000B8A1A4402814B8A1A444281898A114499
:10831000818143F6FF71C18170470000F0010020A8
:10832000084940F61C72B1F90C00904202DA00F5DF
:108330009F7005E041F2E302904201DDA0F59F70DD
:10834000C88170474C00002038B51348C16941F01E
:108350000401C1611E208DF8000002208DF801008B
:108360008DF8020001248DF803406846FDF714FAE9
:108370000A4984200880094947F690602C3108801A
:108380000020091F0880054914310C80091F08804E
:10839000081F048038BD00000010024000080040A3
:1083A00030B420491E4A45788B7A114692F83B40FA
:1083B00091F83910AC4218D14BB10379994202D0EF
:1083C0004379994201D140791AE0807909E08379B3
:1083D000994202D0C479A14202D182F82F3011E033
:1083E000407982F82F0030BC7047C578AC42FAD192
:1083F0006BB1C379994202D0037A994205D1007AD0
:1084000082F82F0030BCFEF793BB407AE9E7437A4D
:108410009942E2D00479A142DFD0007AE1E700007E
:108420005C04002038010020FEE700002DE9F04741
:108430000446007F012868D13548E1880288511A36
:1084400089B2072916D30088E080B4F9000044F20D
:10845000DD414843401346F6D96148438013A0608C
:10846000401000B2A0814FF08051B1FBF0F0F7F75F
:10847000DDFF2061B4F90C6096B1B4F902104DF63D
:10848000B05048430014A082B4F904704DF6B052C5
:1084900007FB02F24FEA2245E58204D4024603E0DC
:1084A0000020E08330E0424212B22283002D01DB43
:1084B0002B4600E06B421BB2DFF85890638398466E
:1084C0004FF4804AB24208DAF7F7A7FF2169F7F7BD
:1084D0007AFEF7F7CEFF801304E0002901DA484660
:1084E00000E05046E083B04509DA2846F7F795FFEB
:1084F0002169F7F768FEF7F7BCFF801304E0002F4F
:1085000001DA484600E050462084BDE8F0870000CC
:108510005807002000C0FFFF2DE9F0414C484D4EA8
:1085200000250078A6F15004022806D14A4FF87BB6
:10853000022802D1B7F8440030B1A5862564B5629F
:1085400084F83850BDE8F08144488168C0684943E8
:1085500000FB0010FBF7EAF840F233314843810B8F
:10856000B4F8440043F6CC42504301EB903080B263
:1085700043F69911A4F84400884209D338481146BB
:10858000B0F90400884203DB97F84A00032813D0AF
:108590000123B4F934101A460020FEF717FAA0861A
:1085A000B4F84000012301B21A460020FEF70EFA8B
:1085B00020648003B06226E0B4F8460041F69A13C6
:1085C000A0F51852663A9A4209D2B4F94400214AF9
:1085D000FAF74CFF2064012084F8380022E044F2CE
:1085E0004711884212D994F83800D8B11D48017853
:1085F000491CC9B20170022914D30570206C10B156
:10860000401E206408E084F838500BE0A0F580405C
:10861000B0F5A47F03D2206C8003B06202E084F83E
:108620003850B562B4F840000A4980B20839323493
:1086300001F010FDB4F90000B4F91810414389139A
:108640006180B4F9161048438013A0807AE70000D7
:108650004F070020900A0020A8020020CC0900202B
:10866000F2050020320100200D480021A32280F8ED
:108670002810C18381865030C2600E22028241F2EE
:108680006202426108220283418341F25552828391
:108690009203C0E9081240F28E3282608162704714
:1086A000400A00202DE9F0410546FBF737F9204C40
:1086B000204E074620686168421C8A4220D009B9D2
:1086C0003F281DD004EB0010AA7A05F10B010E30F3
:1086D000F7F759FD2168686804EB0111886021688B
:1086E000A87A04EB0111888172B62068401C2060D2
:1086F000402801D30020206062B6307888B114E0B1
:108700003846FBF7F3F80A28D4D3706800F070FA03
:10871000002109A001F0D0FA70604FF0FF30BDE8F1
:10872000F08155203070F9F71BFC0020F7E70000BE
:10873000B8140020580800206465765F63616E31CC
:108740000000000010B504000B462D4AC3F10000E4
:1087500028D56442002B12DAA04207DA214600F045
:10876000F1FB32F81000C0F5404041E001462046E0
:1087700000F0E8FB32F8100000F5004038E0A342BA
:1087800008DA2146184600F0DDFB32F8100000F54B
:1087900040402DE0204600F0D5FB32F81000C0F537
:1087A000803025E0002B12DAA04207DA214600F0E3
:1087B000C9FB32F8100000F5804019E00146204660
:1087C00000F0C0FB32F81000C0F5004010E0A342FA
:1087D00008DA2146184600F0B5FB32F81000C0F563
:1087E000804005E053B1204600F0ACFB32F81000A9
:1087F000B0F5004F01DDA0F5803010BD002010BDA8
:10880000E0B2000840438013494300EBA13000224E
:108810000302002B14DDB3F5001F01DC802001E012
:108820004FF4005093FBF0F1014401EBD17149107A
:10883000814206D0521CD2B20846062AF2D300E08A
:108840000021C80000B2704702E008C8121F08C12A
:10885000002AFAD170477047002001E001C1121FC1
:10886000002AFBD1704700002DE9F047BD4CBE48FF
:1088700021880288511A89B20F297DD30088A4F17A
:108880003C052080288F08B1401E28872B78B74AE6
:10889000C3F3810001281ED0022821D0118BB148DA
:1088A000B44EDFF8CC92407EB6F806C00027B1F592
:1088B000926F1CD8142818D3782060764CF01000E2
:1088C000F08040F26660A88123F001002870D77321
:1088D00089F8007018E0108B00EB4000C00302E044
:1088E000108BA5494843010CD9E7401C04E0B1F5C1
:1088F000216F09D910B1401E607605E02CF0100000
:10890000F08043F001002870B5F90200B5F9143089
:108910004143C3EBC303C1F38F31C3F3D10303EB73
:10892000510109B2A9829046128B4FF080535043F7
:10893000B5F91620C0F38F30C2EBC202C2F3D102E8
:1089400002EB500000B2E882AA6A42431213EA62C4
:1089500093FBF2F22A63894A1080A2680A44A2605B
:10896000E1680144E160207C401CC0B2207407280B
:1089700002D942F3CF0000E0E8E02883C910698300
:10898000E760A76041F6C8012774884204DD2A8B9E
:108990007B49B1FBF2F1E981C117890341EA9041BA
:1089A000800342F69B420023F7F7BCFBA8846D4886
:1089B0002A78A0F13C009307B0F90600C2F38102C7
:1089C00000EB801101EB003141F30F3115D5012A85
:1089D00007D0022A0BD04EF6AC3141430914A180D6
:1089E00011E049F2586250430014A08020E04CF29C
:1089F0000C3141430914A18026E0012A0ED0022A3D
:108A000018D0A08069845F4948430014A4F81E0070
:108A1000FAF754FA5C480088C0B143E04AF2904249
:108A200042431214A2804BF2C822504300146884BF
:108A3000E183EDE74CF6345141430914A1804DF632
:108A40006C314143091469845049DDE795F82000F1
:108A500000BB88F80F7089F80070B5F91A00A0F50E
:108A600014512C39B1F56E7F18D2617FF42912D9D7
:108A70004749E880434AA1F8460050430014A880C3
:108A8000A1F84400FF2085F8200081F82800414922
:108A90003C20087006E0491C617703E0607F08B164
:108AA000401E6077B5F91A00B4F91E203A49904289
:108AB0000DDDA27E7D2A08D9F28842F00802F280FC
:108AC0000A7822F002020A700EE0521C06E0A2F2BE
:108AD0003D12904208DAA27E12B1521EA27603E045
:108AE000F28822F00802F280B4F90420904214DAED
:108AF0002A4B9B68B3F5FA7F0FDAE07E3E2809D94E
:108B0000F08840F01000F0802777087820F002000D
:108B100008700CE0401CE07609E002F23D12904241
:108B200001DD8888A0B1207F08B1401E2077B5F90B
:108B30001810606908446061217E491CC9B2217621
:108B40001F2903D94011A88367612776BDE8F08704
:108B5000207F7D2804D9F08820F01000F080E6E71F
:108B6000401CE3E71005002058070020A802002061
:108B70004F070020100C002030330100800B002034
:108B800074E8260B188601005A070020E03801001F
:108B9000680E00204C070020F20500204005002050
:108BA000024941F2F460886270470000D40400205A
:108BB00070B50D4C207828B1012808D0062505286D
:108BC0000FD10BE00948F9F745FC012004E0074804
:108BD000801DF9F73FFC0520207070BDF9F75AFCA5
:108BE0002570257070BD000050070020E8B1000816
:108BF0000A4A4FF0FF31B0EBA20F0CDA00280ADB73
:108C00000749096851F820004068006900B1004731
:108C10006FF0050070470846704700000400000030
:108C20008C08002070B50A4DA86870B1002409486E
:108C3000AC60F8F71DFB084804604460A0F5816053
:108C4000046044602C70002070BD6FF0040070BDA3
:108C50005808002000640040B81400207FB5054685
:108C60000024631E244A4FF00050072D41D2DFE854
:108C700005F04004111E21403C00814208D2D0681A
:108C8000202805DA1D4B43F82010401CD0600CE072
:108C90001C4627E08142FBD210692028F8DA174BE6
:108CA000803343F82010401C10610023F0E7F8F7F0
:108CB000F5FA17E000208DF80B000121ADF8000057
:108CC0000422ADF80400ADF808008DF80C108DF802
:108CD0000A00ADF80220ADF806208DF80D106846A8
:108CE000F8F718FB204604B070BDBDE87F40FAF7E6
:108CF000A9BE1846F7E7000058080020C018002059
:108D0000F8B5414EB06801287BD04048F8F7B0FA7A
:108D100001210820FDF784F801210846FDF780F8BD
:108D200001214806FDF764F801214FF4EA10FAF733
:108D3000A1FD4FF48070ADF8000003248DF80240CF
:108D40000420334D8DF8030069462846FAF740FDAC
:108D50006815ADF800008DF8024018208DF803006A
:108D600069462846FAF734FD14208DF800000227E2
:108D70008DF8017000248DF8024001258DF8035014
:108D80006846FCF709FD13208DF800008DF801708E
:108D90008DF802508DF803506846FCF7FDFC162054
:108DA0008DF800008DF801408DF802408DF80350D9
:108DB0006846FCF7F1FC17490120FFF74FFF164901
:108DC0000120FFF74BFF15490120FFF747FF14492A
:108DD0000120FFF743FF13490120FFF73FFF002168
:108DE0000320FFF73BFFF8F7EFF90F4804604460FA
:108DF000A0F581600460446034700020B560F8BD67
:108E0000FFE74FF0FF30FAE7580800200064004009
:108E1000000C014020FF401820FF431820FF441899
:108E200020FF451820FF2518B81400202DE9F04731
:108E300081461E4886B0174680680E46A0B14FF0A6
:108E4000FF381FB36846FAF70BFE401C0ED00DF139
:108E50000B019DF80A208A464846019DF7F793F9D1
:108E60009DF80A403D601DE06FF0040006B0BDE8CB
:108E7000F08700BFFAF7E6FD411C15D0A84213D1D8
:108E80006846FAF7EDFD0198A84201D04046EDE7AB
:108E90009DF80A2009EB04005146F7F774F99DF894
:108EA0000A000444B442E5D32046DFE75808002016
:108EB0002DE9F0470646224886B00024806888B134
:108EC000601E002A10D012680192B2F1005F0BD22E
:108ED000CF0801F007054FF000084FF004094FF0EC
:108EE000080A17E06FF0040006B0BDE8F08700BF85
:108EF0008DF80AA08DF8089006EBC4008DF8098063
:108F00000168CDF80B104068CDF80F006846FFF7F8
:108F1000C9FB641CBC42EBDB7DB18DF80A508DF8B7
:108F200008908DF8098006EBC4012A460DF10B006C
:108F3000F7F729F96846FFF7B5FB0020D4E70000F2
:108F400058080020090A05D0B0FBF1F0FF2800D92D
:108F5000FF20704700207047D0E90021C368521AF3
:108F60005A4301EBA231816041607047B0F90020A3
:108F7000B0F90210B0F90630521A5A4301EBA2318F
:108F8000818041807047000030B5494B18884949BD
:108F90008A89801A85B24848484A0F2D047801F121
:108FA0004C001DD31D888D81117A090713D5022C21
:108FB00001D0434912E0434DB0F90210B5F9005019
:108FC000A94205DC02DA01F1020108E0458007E070
:108FD000A1F1020103E0022C02D13B490988418042
:108FE000B0F840101D88691A89B29C2949D31988A4
:108FF000A0F84010D16A0023B1F5804F31DB33492E
:10900000096DB1F5405F2CDD314940F26665B1F97B
:109010001010A94212DD43F69915A94202DB40F275
:10902000333108E040F23335A1F26661694343F21F
:10903000333591FBF5F1A0F8441001E0A0F844307D
:109040002449B2F80A510978C1F381012DB100BF5A
:10905000B0F8441001F21E511CE092F84A20032A95
:1090600010D0A0F84430022C01D0A0F84430B0F960
:109070005C10B0F9443001F114029A420DDAA0F804
:109080005C2030BD012901D00229E1D1B0F84410A3
:1090900001F23331A0F84410E5E703F114029142E4
:1090A00003DD1439A0F85C1030BDA0F85C3030BD91
:1090B00058070020000000204F070020A8020020D1
:1090C000D2040020D0040020CC040020380100206D
:1090D00040050020D40400202DE9FC41012102209C
:1090E000FCF786FE01211920FCF79AFE01213C487D
:1090F000FAF7C0FB4027ADF8007003248DF802405A
:109100000420384D8DF8030069462846FAF760FBC5
:10911000E001ADF800008DF802401C208DF803003E
:1091200069462846FAF754FB4FF4E0712846FAF7EF
:10913000D6FBA815ADF800008DF8024010208DF880
:10914000030069462848FAF743FB4FF4A060FCF798
:1091500055FB1D208DF8040001268DF805600025C3
:109160008DF806508DF8076001A8FCF715FB1F4924
:109170008C2008801D494FF6FA702C3108806E2033
:10918000091F0880194814300680184808300780E5
:10919000164920310D80154AD020121D1080134A27
:1091A00045F2F300183210800A1F45F2500010807B
:1091B0000E4A4FF6FF7038321080121D1080121DBB
:1091C000108041F21B10088000F012F8FAF76CFED4
:1091D000064810300580001F0480BDE8FC810000B7
:1091E000000C1A0000100140000C01400004004077
:1091F00070B51D20FCF7A3FA2B4D4FF48071284663
:10920000FAF764FB840080212846FAF75FFB44EA02
:10921000400440212846FAF759FB0443E0B2234CAE
:1092200084F83C00FAF7FCFB0546052805D92048E0
:10923000C18841F04001C18001E084F838501D48E8
:10924000007A000703D594F838001B490D5C4FF6EF
:10925000FA702063E062A06260622062E061A06157
:109260001648606300206064206584F83F0084F83D
:109270004000FAF783FBA07AFF2812D05FF00200CB
:1092800084F83D000E480088A0662846FBF770F879
:10929000207820F001002070BDE870401D20FCF710
:1092A00064BA0120ECE70000001001403801002002
:1092B000100C0020A8020020DCBB0008DCFF050029
:1092C000240400402DE9F0475248534902880B8896
:1092D0009A1A92B20F2A69D30988DFF84091018067
:1092E000B9F81E10027D00EB42029180017D491CFD
:1092F000C9B20175082959D3002404752246017D9D
:1093000000EB4103491CB3F90430C9B202EB63021C
:1093100012B201750829F2D341490475414B4A80C4
:1093200044800E789D895FEAC67C40F6386A4FF02B
:10933000030714D0A2F22B5C42F6E858C44520D3B0
:10934000A1F1020C26F00204ACF8002047750C7065
:1093500040F22B54A24211DA45F004021EE046F01E
:1093600001060E70524507DD45F001029A8126F094
:1093700002020A70477517E0447515E045F00202D5
:109380000CE052450CDA8775427D12B1521E4275CF
:109390000AE046F002020A7025F007029A8103E013
:1093A000837D2BB15B1E837540888880BDE8F08784
:1093B00042F6AA239A4229DAB1F904502DB941F2B2
:1093C000CD039A4201DA4480EEE7174B920302EB99
:1093D000833241F67243B2FBF3F212B2428099F843
:1093E00008400346240702D540F2333401E040F63A
:1093F0009914A24200DA5C80B3F90220521B02F5F4
:10940000A372B2F5237FCFD85D80CDE74FF48043C0
:109410004380C9E7A40C002058070020A8020020C0
:10942000F2050020100C0020C8F1FFFF2DE9F041EB
:109430006D4CDFF8B8E14FF0000594F83410C80720
:1094400006D094F938104B42002958DD0E4657E0FB
:10945000674884F83750A4F84250664A90F83800BC
:1094600084F840009586CEF80450CEF80850624E3D
:1094700040F26663CEF80C50A4F87C3036F8100049
:109480005E4E768830444FF6FF7606EA800024F878
:10949000300B4FF0806044F8040CA32020846084DB
:1094A0005810A084E38440F6991020855800608508
:1094B0004FF48050A08541F23330E08541F2666080
:1094C000208641F69910608641F6CC40A0864FF484
:1094D0000050E08642F23330208742F266606087B7
:1094E00042F69910A08742F6CC40E08782F8A1505E
:1094F00041F00100207184F84450BDE8F0811E461F
:1095000094F937004242002801DD074600E0174683
:10951000F61B012E0BD0002800DB02465FFA82F614
:1095200084F8380094F84F00012805D041E0002964
:1095300000DA1946CEB2F3E794F939305942002BDC
:1095400001DB184600E0084694F93A20C7B25042C1
:10955000002A01DB944600E08446BC4508DD002A71
:1095600000DA0246D7B2002B00DA0B46D8B207E089
:10957000002B00DA0B46DFB2002A00DB1046C0B237
:1095800004EB4000B0F9501004EB470030F9502FC5
:1095900011444910018084F84F5084F83E5084F8FB
:1095A0003D5084F83C5084F83B5084F83A5084F89D
:1095B000395004EB46007546B0F9500024F8420FCC
:1095C000BEF80410C82309B26422FDF7FFF96860F1
:1095D000E968401AA9680844A860B5F90010484332
:1095E000C013E860608788E7240C0020E0050020B5
:1095F00038010020A8020020EEBB00084C0000202B
:10960000F0B4544890F83410C90776D0524990F815
:109610004030002291F838108B426FD04F4CA0F8A8
:1096200072204F4DE65C04468E4294F9374002D0DA
:10963000EE5C8E420FD1641C64B280F83740EB5C64
:109640008B4202D1641C80F8374090F937300F2BE1
:109650001BDD0F2317E0434DEE5C434D8E4202D0DD
:10966000EE5C8E4211D1641E64B280F83740EB5C30
:109670008B4202D1641E80F8374090F937406FF07A
:109680000E039C4201DA80F83730324B90F83F509D
:10969000393390F83740EC5490F83F305B1CDBB224
:1096A00080F83F30062B01D380F83F2090F93940F5
:1096B00090F93B309C420ED190F93D40A3420AD133
:1096C00090F93A4090F93C309C4204D190F93E40E8
:1096D000A34200D1012280F84F201F4A80F8401099
:1096E00090F937501378214A012D0DDD14465E079D
:1096F000A46804D544F0080403E028E015E024F051
:109700000804946080F83510B5F1FF3F0ADA5B0772
:10971000936802D523F0080301E043F00803936047
:1097200080F83510F0BCFAF729B990F84F100129EC
:109730000DD1B0F8721043F60953491C89B2A0F854
:109740007210994203D9A0F8722080F84F20F0BC23
:1097500070470000240C002038010020D0BB000816
:10976000D6BB0008E2BB0008E8BB0008A802002046
:1097700010B502884188B0F90830114409B281FB64
:109780000313890B428041EA8341B0F90420B0F908
:10979000063082FB0332940444EA93321144818000
:1097A00010BD000030B52049204AB1F86A30108859
:1097B000C01A80B20F2836D31088A1F86A001C4D59
:1097C00000204FF000432A5C940903D00124B4EB3D
:1097D000921F24D1D20622D0164A52F820201268B5
:1097E000134C123434F81040224201EB000494F977
:1097F000722008D00A2A04DB0A6823FA00F4224304
:1098000008E0521C09E012F10A0F05DC0A6823FA8D
:1098100000F4A2430A6002E0521E84F87220401C49
:10982000C0B21128CFD330BDF80500205807002062
:10983000E4B60008E4B700082DE9F0077A497B4850
:109840000A8903889A1A92B2082A75D30088088177
:10985000A1F12C0042890AB1521E4281744A92F849
:109860002820802A68D302F03F020A70C2890AB118
:10987000521EC281B1F90620902A0CDB8A46FF2ACB
:1098800009D08146C089002856D16A480023007853
:10989000092805D005E0BDE8F007634800F0BEB92F
:1098A0000823654A92F8EE500DB143F00403634873
:1098B000817AC90701D043F00203D2F808C05FEAF9
:1098C0000C5101D543F00103176800215C4EFC03E5
:1098D00002D596F8654004B18021C4885FEA4468E7
:1098E00001D541F040015FEA845801D541F02001E3
:1098F0005FEAC47801D041F01001007A400701D539
:1099000041F008014F480078C00701D041F0040140
:10991000A00601D541F001010020012D00D1082051
:1099200096F870508DB992F84A20032A05D0022A81
:1099300006D0012A07D008E072E040F0030004E0FE
:1099400040F0020001E040F001007A0701D440F04D
:109950002000CCF3C0020025CCF3002C624502D1DC
:109960003A0700D4042596F86F20012A01D145F06A
:109970000105354A0027BC4612783E46C2F38102F3
:10998000012A04D0022A04D0032A04D004E00226CB
:1099900002E0042600E010262C4A64060ED5224C74
:1099A0001C342478240609D51478640606D4284A81
:1099B00040F6CC44926D6243140C05E0B2F8B62038
:1099C00040F699146243940B4FF008088AF80A8015
:1099D0004FF061088AF80B808AF80C308AF80D1075
:1099E0008AF80E008AF80F508AF81070270A4B4048
:1099F00083F06901414069408AF8117079408AF822
:109A00001240614052468AF813C071408AF81460CF
:109A100051754FF4C871A9F80E10FF20AAF806007E
:109A2000BDE8F00770470000040700205807002039
:109A3000F80500204F070020A8020020100C00208D
:109A4000680E0020C00A0020D40400203801002045
:109A5000640900205B48816941F0FC0181614FF499
:109A6000A060FBF7CBFEFAF7AFFAF7F7D5F8FBF7F4
:109A70003DFD002154A000F01FF956490860FDF794
:109A8000B7F8FCF7A9FEFFF727FBFBF79BF9FFF7F9
:109A9000AFFBFAF709FA504D4FF40050A5F81A0140
:109AA0004E480078FF2801D0FCF762F8FCF716F862
:109AB00000214FF4FA5340F2EE220020401C80B205
:109AC0009842FBD3491C89B29142F6D34448002600
:109AD00080F87260F6F730FFF8F7B4FDF8F7B6FAE1
:109AE000FEF732FC10223F493F48F6F74CFB01F0ED
:109AF000FFF93E4C3F4FE08820F04000E0803C48BA
:109B0000017821F020010170FA20F8814FF496705D
:109B1000A5F84200FFF744F837493848FBF789FFBA
:109B20003748FBF7ABFF3748416A88473648416BF7
:109B30008847FEF799FD3548F9F7BCF9F8F7B8FA08
:109B400033494220C8803349C8603348F7F710FAD8
:109B5000A86820F48070A8603E71E088E0812089C8
:109B6000208260896082F9F795FDF9F7F1FCFEF734
:109B70007BFE01F03DF9FFF7A5FB00F039FAFFF796
:109B800011FE00F0E9FFFDF79BFEF9F7A5FAF8F7E3
:109B9000B9FAFAF70BFCFFF7F7F9FCF7D1F9FAF786
:109BA00029F8FAF75BF800F0B5F8FFF745FE17481B
:109BB000F9F72CF800F0A8FAFCF752FEF9F7B0F923
:109BC000CBE70000001002406465765F63616E3190
:109BD000000000005C080020A802002001E8010845
:109BE00040050020680E002038060020100C0020E0
:109BF000380100204C070020100A0020E009002056
:109C00001004002020000020CC0000204C0B00207D
:109C10004007002044040020C00B0020F0B5234979
:109C20000278B0F9064000231F4E31F81210FF2CC5
:109C300018D0B0F904701E4DBC4231DA00EBE407D5
:109C400004F00704BF7AA7408478FFB23CB190F8D3
:109C500001C0ACF1010C64451FDA3C061DD455F877
:109C600022200DE056F82220116012498A79521CF8
:109C7000D2B28A71022A02D38370C3808B71F0BD85
:109C800011608178491CC9B2817042789142F6D343
:109C90008370C188491CC180F0BD56F82220EFE7CF
:109CA00055F822201160F4E7C4B80008F6B60008A1
:109CB0006CB80008D80600202DE9F0410F46804618
:109CC0000024124D124E08E0286850F82400016864
:109CD0004046F6F76AFA38B1641CB4EBA60FF3DB22
:109CE0006FF00100BDE8F081286850F8240040685A
:109CF000016829B13846884728B16FF00200F1E7C2
:109D00006FF00500EEE72046ECE700008C0800202D
:109D100004000000F0B561486149B0F86C200B8880
:109D20009A1A92B29C2A7BD30988A0F86C105D49DC
:109D30005D4F91F82A1001F0070297F84A10022AA5
:109D400000D1491E594C80F83E104FF00203E288C2
:109D50004FF00001550401D5012236E0A489E50643
:109D600001D5062231E0250701D508222DE0550650
:109D700003D44F4D2D78AD0601D5042225E01505FD
:109D800001D5072221E0150601D50A221DE095061E
:109D900001D50C2219E0150701D50B2215E0550756
:109DA00001D4D50501D510220FE0D50601D5052235
:109DB0000BE0650703D4A50701D4E40702D080F8BF
:109DC0006E3007E0920403D5032280F86E2001E094
:109DD00080F86E10374A384C92F820E0324A251F3E
:109DE000D2F808C02D4AB2F87060721C92B2BEF16F
:109DF000000F0DD02CF4000CC7F808C090F86E705E
:109E0000B7B11E2F1AD090F86F200AB325E007E0F3
:109E10004CF40006BE60A0F870200A2A01D223602C
:109E2000F0BD142A01D22B60F0BDA0F87010F0BD77
:109E30002B60A0F8701080F86F10F0BD642E04D273
:109E4000A0F87020322AEED3E9E7A0F87010EAE714
:109E50007F1C80F86F70A0F8701090F86F20012AB6
:109E600010D0002AE9D0B0F87060761CB6B2A0F825
:109E700070601E2ED7D323603C2EDED9521E80F890
:109E80006F20D2E7B0F87020521C92B2A0F8702078
:109E90002360C82AD1D980F86F10C6E7F8050020E2
:109EA00058070020680E0020A8020020100C002097
:109EB00038010020D4040020141C0140F0B54548AE
:109EC000B0F84810491C89B2A0F8481002297DD387
:109ED00041490024A0F848400A78404B042A5BD04E
:109EE0004FF48041082A0BD0A0F11002B2F90020F3
:109EF0008A4200DA1146B3F984208A4200DA114618
:109F0000374A12698A4200DA11B2418282881D8A78
:109F1000C2EB8502334D12B22D78C5F381062D4D6B
:109F200040F6D9467243B5F9765092126A4312133D
:109F3000C26086681546C6EBC60642F3D102F60239
:109F400002EBA6328260C66C1644C664B0F850704C
:109F50007F1CBFB2A0F85070B7F5806F04D3B61263
:109F60000682A0F85040C464C66A891AA6EB461758
:109F700040F2545207EB07174A43A7EBC61602EB11
:109F80004602466A32444262B3F93430B2EB034FC0
:109F900006DD1A04426206E01349B1F90410AFE786
:109FA000002A00DA4462C162104990F83D2091F81D
:109FB00038108A420DD080F83D10B0F84210A0F859
:109FC0004410B0F84010A0F8421000E001E0A0F802
:109FD0004050F0BD400500204F070020A80200209F
:109FE000080E0020D40400201C0E002038010020A0
:109FF00015481649B0F85A200B889A1A92B20F2ABF
:10A0000020D30988A0F85A10B0F900104FF480420C
:10A01000C1EBC12141F35131A0F86C100C490B7810
:10A02000A0F11001022B06D1B1F90030934202DAFF
:10A030001B1D0B8000E00A800021A0F8601020F8B2
:10A040005C1F428070470000400500205807002038
:10A050004F0700204FF6FF7202EA800210F44043DF
:10A0600015480ED0B3F5804F14D0B3F5004F4FEA2A
:10A07000122216D0C2F5807330F813305B424B8049
:10A0800005E0120A30F812304B80C2F5807230F8C9
:10A0900012000FE0120AC2F5807330F813304B80C3
:10A0A00005E030F81230C2F580725B424B8030F828
:10A0B0001200404208807047E0B40008104A518AFC
:10A0C000D08A928A16384639A2F1110200D5494247
:10A0D000002A00DA52421144002800DA40420844C3
:10A0E000084943F6284300B2B1F936205A43921387
:10A0F00040F2D733584302EBA030C88670470000C7
:10A10000A802002040050020F0B5904990480A8937
:10A1100003889A1A92B23E2A1ED30088088101F160
:10A1200038004FF4FA63428A9A4202D2521C4282A9
:10A1300000E04382874A92F82220802A0CD302F062
:10A140003F020A70B1F90620402A06DBFF2A04D03C
:10A15000C2883AB1521EC280F0BDBDE8F0407B48D3
:10A16000FFF75CBD428A9A42F6D307784FF0010EA2
:10A170003A074FF0FF055BD5847A40F2DC52630763
:10A1800008D444F004038372C28081F80BE081F8A4
:10A190000AE04CE04378072B05D0032B03D0052BB6
:10A1A00001D0062B07D1660605D444F04003837224
:10A1B000C280052239E0654A5FEA437C02F1380239
:10A1C0004FF42076127A0DD55FEAC26C0AD45FEAAA
:10A1D000446C07D442F0100202723A0628D4C680BA
:10A1E000192222E0DF0709D0970707D4670605D4B4
:10A1F00042F002020272C680042216E09F0709D5CF
:10A20000170707D4670605D442F008020272C68019
:10A2100003220AE01B070BD5530709D4630607D4B2
:10A2200042F004020272C6800B22CA728A72CD808A
:10A23000494AB2F92230B2F91A7003F23D140022F1
:10A24000A74200DB0276414E444C06F13806A47961
:10A25000B6895FEAC46C06F101064FF4C874B6B261
:10A2600013D58681B6F57A7F05D9017A21F0800170
:10A2700001728281F0BD037A1E06FBD4828143F015
:10A2800080020272C480112035E09F4216DA037EFC
:10A29000052B13D28681B6F5487F04D98281027AD4
:10A2A00022F040020272027A5606E3D45B1C037667
:10A2B00042F040020272C48002201CE0284B1C893C
:10A2C000C4F3C006C4F3002740F2EE24BE4216D108
:10A2D0001E78360713D4427E012ACBD1428BB2F5C9
:10A2E000167F02D2521C4283F0BD827A42F00202F3
:10A2F0008272C4800F20C8728872CD80F0BD93F83E
:10A3000011714FF40046012F18D1164F41F6583CF9
:10A310007F6C674512DD83F810E1134B1E60C38A22
:10A32000A34202D25B1CC382F0BD4FF4FA73C38018
:10A330001C23CB728B72CD80C282F0BDC2820A48D0
:10A3400083F81021001F0660F0BD0000E806002021
:10A3500058070020F8050020D4040020100C00202D
:10A36000A802002038010020140801402DE9F05F08
:10A37000DFF8FCB3FF489BF81830011D0A1DFE4CA6
:10A38000012B5FD0B4F85E300380B4F86000088021
:10A39000B4F862001080FDF725FBDFF8E083F84D8C
:10A3A00049F2CD32B8F91E00A883B8F9201043F65F
:10A3B000CC4C00EB410151430914E983B5F922303B
:10A3C000B5F9206001FB03F200FB062242F38F3255
:10A3D0006A82B5F91870714307FB0CF740F2333C01
:10A3E000BF1302FB0CF207EBA23200FB13102A830F
:10A3F00040F38F30A882B5F91A1043F6AE7251437C
:10A4000000EB0012891302EB8010DE4F01EBA0304D
:10A41000DD4E6883786C3060316930468847DB49AF
:10A42000308948800846FDF7BFFBD94E4FF0000940
:10A430004FF0010A307808280DD0698F298204284E
:10A4400033D01BE0B4F864300380B4F866000880B1
:10A45000B4F868009EE7CF4890F93710491C0229EC
:10A4600021D890F8741019B1B5F85A00288205E087
:10A47000698F2982A5F85A1080F874A0B5F91410D4
:10A48000B5F90A00C44AF8F765FAE862B4F91A1196
:10A49000884204DDC048E962027C914081623078E4
:10A4A000042816D00CE0688FE0E7D8F824000014E8
:10A4B000E862E07B04280CD0C5F82C9086F8009068
:10A4C000B54AB5F91210B5F90800303AF8F742FA72
:10A4D00002E0B87AF0B3B148A862A94DAE4E443E4E
:10A4E000A86A3060E86A706030461035FBF704FDFA
:10A4F0002888A5F14C01FFF7ADFDA5F15C08D8F85F
:10A500001010C8F86C10B5F91020B068B5F9121029
:10A5100000FB02F7F368484303FB117646F38F37DD
:10A5200003FB0200AF8740F38F36EE879C4D284631
:10A530006F80AE80FDF77AFF287F08F114050128AF
:10A5400033D0704242104DF6B35047436A803914FD
:10A55000298000E026E04046A8F8006053184380B8
:10A56000511AA8F8041084F80C90B8F90030002BA8
:10A5700001DD84F80CA0B8F90200002802DD217B7F
:10A58000891C2173B8F90420002A02DD217B091DF2
:10A590002173217B072920D2DFE801F01F1B34182B
:10A5A000301D32004FF4AF7096E77D48B0F920308F
:10A5B00059424A106A80B0F91E004DF6B351484323
:10A5C000011429804046A8F80030C7E784F80DA0A0
:10A5D00003E0022100E003216173DFF8A4A1714EC2
:10A5E000714F9AF800100129617B0DD0072972D2B2
:10A5F000DFE801F071FCFBFAF9F8F7000421EBE762
:10A600000521E9E70621E7E70729F0D2DFE801F0B5
:10A6100063042F6489D5EF0001461846FBF7F0F973
:10A620002860B5F9020040F68151484381136980E2
:10A63000B5F9000040F681525043801328800A1873
:10A64000A2F68152B8F80A305242C3EB620212B24B
:10A65000A8F80820002A01DCA8F80890B8F808201B
:10A66000A4F862201144A4F8601008446DE140424F
:10A6700001B2504200B2FBF7C3F92860B5F90200FD
:10A6800040F68151484381136980B5F9000040F6D6
:10A6900081525043801328800A18A2F68152B8F8DC
:10A6A0000A305242C3EB620212B2A8F80820002A14
:10A6B00001DCA8F80890B8F80820A4F8622011443A
:10A6C000A4F85E1008446EE13046F6F703FB012360
:10A6D0001A460721CAE0D4E019461046FBF790F964
:10A6E0002860B5F9020040F6815148438013688024
:10A6F000B5F9001040F68152514389132980421860
:10A70000A2F68152B8F80A305242C3EB620212B28A
:10A71000A8F80820002A01DCA8F80890B8F808205A
:10A7200068E15942404209B200B2FBF769F928607A
:10A73000B5F9020040F68151484380136880B5F9AD
:10A74000001040F681525143891329804218A2F625
:10A750008152B8F80A305242C3EB620212B2A8F832
:10A760000820002A01DCA8F80890B8F8082071E158
:10A770004C0B0020342C0140A80200204005002092
:10A780004C00002038010020440400200004002078
:10A790004F070020240C0020100A0020A2FEFFFF1B
:10A7A000800B002000240140002801403046F6F7CD
:10A7B00091FA01231A46052158E01146FBF720F9CA
:10A7C0002860B5F9020040F6815148438013688043
:10A7D000B5F9001040F6815251438913298042187F
:10A7E00006E076E14AE11BE1ECE0BCE08FE010E03E
:10A7F000A2F68152B8F80A305242C3EB620212B29A
:10A80000A8F80820002A01DCA8F80890B8F8082069
:10A810004BE1504201B2584200B2FBF7F1F8286018
:10A82000B5F9020040F68151484380136880B5F9BC
:10A83000001040F681525143891329804218A2F634
:10A840008152B8F80A305242C3EB620212B2A8F841
:10A850000820002A01DCA8F80890B8F8082052E186
:10A860003046F6F737FA01231A4606213846F6F73E
:10A8700031FA01213046F6F7A3F901213846F6F7FF
:10A880009FF9BAF80800ABF80000BAF80A00ABF874
:10A890000200BAF81000ABF8040055465E46AB481B
:10A8A000F8F716FAB4F85E00F1880844A4F86400DA
:10A8B000B4F8600031890844A4F86600B4F8620076
:10A8C00071890844A4F86800317EA148012978D034
:10A8D00034F85E1F018061884180A18881809C4995
:10A8E000028808310A8042884A8080888880984897
:10A8F000896A0830884795F83E0000287ED0F7F72F
:10A90000C9FD15F83E0F401E2870BDE8F09F0146B6
:10A910001846FBF775F82860B5F9020040F681513A
:10A92000484380136880B5F9001040F681525143C6
:10A9300089134218A2F68152524252082980A4F883
:10A9400062201044A4F860000844A4F85E000021CE
:10A950003046F6F735F900213846F6F731F901238C
:10A960001A460621B0E6404201B2504200B2FBF75F
:10A9700047F82860B5F9020040F68151484380133A
:10A980006880B5F9001040F681525143891342188E
:10A99000A2F68152524252082980A4F86220104443
:10A9A000A4F85E000844A4F8600000213046F6F7E1
:10A9B00007F900213846F6F703F901231A46052165
:10A9C00082E6B4E019461046FBF71AF82860B5F99C
:10A9D000020040F68151484380136880B5F90010A9
:10A9E00040F68152514389134218A2F681525242D5
:10A9F00029805208A4F85E20104400E09AE0A4F8F0
:10AA000062000844A4F8600000213046F6F7D8F848
:10AA100000213846F6F7D4F801231A460721C5E687
:10AA20005942404209B200B2FAF7EAFF2860B5F98C
:10AA3000020040F68151484380136880B5F9001048
:10AA400040F68152514389134218A2F68152524274
:10AA500029805208A4F85E201044A4F8600008443D
:10AA6000A4F8620000213046F6F7AAF80021384623
:10AA7000F6F7A6F801231A46062197E61146FAF7DB
:10AA8000BFFF2860B5F9020040F6815148438013AA
:10AA90006880B5F9001040F681525143891342187D
:10AAA000A2F68152524229805208A4F86020104434
:10AAB000A4F85E000844A4F8620000213046F6F7CE
:10AAC0007FF800213846F6F77BF801231A46052166
:10AAD000C6E6504201B2584200B2FAF791FF286030
:10AAE000B5F9020040F68151484380136880B5F9FA
:10AAF000001040F68152514389134218A2F6815248
:10AB0000524229805208A4F860201044A4F8620040
:10AB10000844A4F85E0000213046F6F751F8002101
:10AB20003846F6F74DF801231A46072198E634F81F
:10AB3000641FCFE607480088A0F5D04168393FF48C
:10AB4000E4AEBDE8F05FF8F7AFBB00004C0B0020AF
:10AB500018000020182C01402DE9F041964C974830
:10AB6000B4F862100288511A89B20F296FD3008895
:10AB7000A4F8620092480088DFF84882C0074FF0CE
:10AB800000054FF0010741D08D4AD4E90C10243262
:10AB90001388B1EB530F02D21288511A08444FF4B4
:10ABA000F371884200D208468749B1FBF0F0616C2E
:10ABB000C1F35101084406466064F5F73CFC0022ED
:10ABC000824BF5F7A4FB4FF04042814BF5F79FFB1A
:10ABD0000E22F5F70BFCF5F765FCA4F8AC0094F831
:10ABE0006D00401CC0B284F86D00082834D3724850
:10ABF00098F84A20001F03789A4201D002704580DD
:10AC0000744A1378744A23B1458021E06564256550
:10AC10006AE0D8F89810A1F5FA618E4211DDE16D75
:10AC20008B1C9E4205DDB0F902100A290DDA491C81
:10AC300006E08E4205DAB0F90210002908DD491E4F
:10AC40004180B0F902000A2802DB177001E0AEE093
:10AC50001570E66584F86D5060484FF4A5420178A0
:10AC6000C1F38101012963D0022964D045F2082192
:10AC70002181A4F8A820B0F9243089B24B439B135A
:10AC8000A4F8A430B0F90E00D4F850C07043B0FB63
:10AC9000F1F35349CCEBCC0C4FEACC2C0988C3F32D
:10ACA000D10303EB9C33B0032365B0FBF1F14D4BB3
:10ACB000C908B3F846C0CCEBCC0C4FEACC2C01EB66
:10ACC0009C31A3F84610F117890341EA964100230D
:10ACD000F5F728FAB4F8AA10C1EBC101C902C008FF
:10ACE00000EB9130A4F8AA00616C206F4218226733
:10ACF00094F87400401CC0B284F87400082805D38E
:10AD0000D008A4F8760084F8745025673648C388C4
:10AD10005A0605D498F80F20022A0FD0A4F88A50BA
:10AD2000254894F83F20B8300C2A2AD2C57429E06F
:10AD300045F6C0519CE744F2506199E794F83820F9
:10AD400094F88E60B2420CD084F88E2094F83D20A6
:10AD500002F00106C2F34002964202D1A4F88A50E2
:10AD600005E0B4F88A2040F6B836B24205D2B4F80D
:10AD70008A00401CA4F88A00D2E743F08002C28017
:10AD8000CEE7C774194B41F2482641F2504C93F874
:10AD90003C400C4B0C2AB3F886300AD3B14208DB96
:10ADA000012C06D0614502DD002B00D18774BDE87F
:10ADB000F0818574FBE7000038010020580700206F
:10ADC00000040040A80200204564BD0100209C4012
:10ADD000133B3340FE030020FF030020D404002077
:10ADE00030010020400A0020100C00204005002007
:10ADF00070B5394C394821880288511A89B23E29E8
:10AE00004DD30088364E20803649307806F114053F
:10AE100018B3488B80002880E96828468847B5F930
:10AE200004003149FCF790FD304A60804FF48045C2
:10AE3000D3884FF000015E0737D4B0F5DC5F2FDD1B
:10AE4000E079401CC0B2E0710A283ED343F40040D0
:10AE500040F00400D080A16036E0888B204A80005A
:10AE6000121D1080888B80005080888B800000B27B
:10AE700090804A8B92002A804A8B92006A80498B8C
:10AE80008900A98018497C31FCF75EFDA080B5F9E6
:10AE900004001549FCF758FD60800120307070BD3A
:10AEA00023F40040A560D0800EE043F4004343F05B
:10AEB0000403A160D380B0F5B45F06DC23F4004046
:10AEC00020F00400D080A560E171D4E9020188423D
:10AED00000DB0846206170BD080E002058070020E6
:10AEE000A4060020A8020020D8BA0008100C0020F8
:10AEF00005494FF48040C860886008610348C188F4
:10AF000021F48271C1807047080E0020100C0020CF
:10AF10002DE9F041404C414E414F207841F2333110
:10AF2000C2074FF000050CD0A28962B394F9070064
:10AF3000002800DA4042C0B2032829D240F2333060
:10AF40002AE0A570E573374AE571A58192F838309B
:10AF5000237220F00800A18040F002002070BD861E
:10AF60007560B560F560116D490005D041F68461EA
:10AF7000A18140F010002070C0B240F001002070AC
:10AF80006574BDE8F081658120F01000207024E038
:10AF9000042803D240F2666060811EE0052802D2D8
:10AFA00040F69910F8E740F6CC42062801D307286E
:10AFB00001D2628111E0082802D24FF48050EBE701
:10AFC000092809D30A2807D341F6CC410B2803D31B
:10AFD0000C2801D342F26661618197F8A10098B90B
:10AFE000B088102301B2B4F90A003622FBF7EEFC58
:10AFF0007060F168401AB1680844B060B6F900109A
:10B000004843C013F060B886B88E10B10120A0701C
:10B01000B7E7A570B5E700001C0E0020C8060020A9
:10B02000A8020020380100202DE9F0414C4C267880
:10B03000F0077CD04B48217A4B4D90F83800814284
:10B0400067D04A4A2346DFF828C1575C93F90E209F
:10B0500093F90730874203D01CF80170874213D15F
:10B0600046F002065B1C26705BB2E3711CF801100F
:10B07000814201D15B1CE37194F90710062901DDBF
:10B080000621E171521C1CE03A4F17F801C03A4FFB
:10B09000844503D017F801C0844513D126F0020679
:10B0A0005B1E26705BB2E371795C814201D15B1E4D
:10B0B000E37194F907306FF005018B4200DAE1711A
:10B0C000521EA273207294F907108A1C042A02D916
:10B0D00041F68462A281234A012912780ADD224BBB
:10B0E00056079B6802D543F0080301E023F00803EC
:10B0F000AB606070B1F1FF3F09DA5107A96802D572
:10B1000021F0080101E041F00801A9606070F8F742
:10B1100035FCA089002630B1401E0004000CA0813F
:10B1200001D1E671A673E87B04280ED000E00CE0A4
:10B13000B5F93410512341220020FBF747FCA886C3
:10B14000002802D1E07B10B1A670BDE8F0810B4869
:10B1500006700B480670207820F001002070F4E79C
:10B160001C0E002038010020A8020020D0BB0008DF
:10B17000D6BB0008E2BB0008E8BB00086C07002053
:10B180004F070020F0B415460D4A0E464FF0FF3130
:10B19000B0EBA20F12DA002810DB0A49096851F857
:10B1A0002000406844682CB129463046A446F0BCD3
:10B1B0001A4660476FF00500F0BC70470846FBE791
:10B1C000040000008C080020173E573CBB3A3E3973
:10B1D000DD379436613541343333353244316130B3
:10B1E0008A2FBD2EFB2D412DCC1C5858586899191B
:10B1F000585858683313005695130054B61300522C
:10B200005A140050FD14004EA115004C4516004A7A
:10B21000761600486C17004672180044BA190042AE
:10B22000741B0040911D003EB420003C9F22003A58
:10B23000E1220038532300368B240034812500326C
:10B240002B2700302028002E5829002CB02A002A55
:10B250009B2C0028D22D00267C2F00242631002292
:10B2600002330020FD34001E5C37001CCC3C001A69
:10B27000873E0018BE3F0016004000140040001238
:10B28000004000100040000E0040000C0040000A8A
:10B29000004000080040000600400004004000029A
:10B2A0000040000001020304050005000102030440
:10B2B0000104000305020000F00100003601000057
:10B2C000F8000000BA0000007C0000007C000000D4
:10B2D0007C000000C91C9C19991CCC199C1CC91924
:10B2E0000000290052007B00A400CC00F5001E01E4
:10B2F000470170019901C201EA0113023C02650293
:10B300008E02B602DF020803300359038203AA0348
:10B31000D303FB0324044C0475049D04C504EE040C
:10B3200016053E0567058F05B705DF0507062F06DD
:10B3300057067F06A706CE06F6061E0746076D07C8
:10B340009507BC07E4070B08320859088108A808CC
:10B35000CF08F6081D0944096A099109B809DE09F0
:10B36000050A2B0A520A780A9E0AC40AEA0A100B36
:10B37000360B5C0B820BA80BCD0BF30B180C3E0CA1
:10B38000630C880CAD0CD20CF70C1C0D410D650D37
:10B390008A0DAF0DD30DF70D1C0E400E640E880EF6
:10B3A000AC0ECF0EF30E170F3A0F5E0F810FA40FE6
:10B3B000C70FEA0F0D103010531075109810BA1007
:10B3C000DD10FF102111431165118711A911CA1158
:10B3D000EC110D122E12501271129212B312D412DD
:10B3E000F41215133613561376139613B713D71397
:10B3F000F61316143614561475149414B414D31486
:10B40000F214111530154E156D158C15AA15C815A9
:10B41000E7150516231641165F167C169A16B71601
:10B42000D516F2160F172C17491766178317A01792
:10B43000BC17D917F51711182E184A186618811855
:10B440009D18B918D418F0180B19261942195D194E
:10B4500078199219AD19C819E219FD19171A311A7C
:10B460004C1A661A801A991AB31ACD1AE61A001BDA
:10B47000191B331B4C1B651B7E1B971BAF1BC81B6B
:10B48000E11BF91B121C2A1C421C5A1C721C8A1C30
:10B49000A21CBA1CD21CE91C011D181D301D471D21
:10B4A0005E1D751D8C1DA31DBA1DD01DE71DFD1D44
:10B4B000141E2A1E401E571E6D1E831E981EAE1E91
:10B4C000C41EDA1EEF1E051F1A1F2F1F451F5A1F0D
:10B4D0006F1F841F991FAE1FC21FD71FEC1F0020B4
:10B4E00000006400C9002D019201F7015B02C00257
:10B4F00024038903ED035204B6041A057F05E3050E
:10B500004706AB060F077307D7073B089F080209DA
:10B510006609C9092D0A900AF30A560BB90B1C0CCF
:10B520007F0CE20C440DA60D090E6B0ECD0E2F0FF5
:10B53000900FF20F5310B41015117611D711381265
:10B540009812F8125813B81318147714D614351526
:10B550009415F3155116B0160E176B17C917261848
:10B560008318E0183D199919F519511AAD1A081BDD
:10B57000631BBE1B181C731CCD1C261D801DD91DF2
:10B58000321E8A1EE31E3B1F921FEA1F4120982095
:10B59000EE2044219A21EF2145229922EE224223D6
:10B5A0009623E9233C248F24E22434258525D725BE
:10B5B00028267826C82618276827B727062854285B
:10B5C000A228EF283D298929D629222A6D2AB82ABE
:10B5D000032B4D2B972BE12B2A2C722CBB2C022DED
:10B5E0004A2D912DD72D1D2E632EA82EEC2E302FF7
:10B5F000742FB82FFA2F3D307F30C03001314131E8
:10B600008131C13100323F327D32BA32F7323433C8
:10B610007033AC33E73322345C349534CE340735A1
:10B620003F357735AE35E4351A3650368536B9367E
:10B63000ED36203753378637B737E9371938493869
:10B640007938A838D738053932395F398B39B73965
:10B65000E2390D3A373A603A893AB23ADA3A013B7E
:10B66000283B4E3B733B983BBD3BE03B043C263CB8
:10B67000483C6A3C8B3CAB3CCB3CEA3C093D273D1B
:10B68000443D613D7D3D993DB43DCE3DE83D013EAB
:10B690001A3E323E493E603E763E8C3EA13EB53E6D
:10B6A000C93EDC3EEF3E013F123F233F333F433F65
:10B6B000513F603F6E3F7B3F873F933F9E3FA93F97
:10B6C000B33FBC3FC53FCD3FD53FDC3FE23FE83F06
:10B6D000ED3FF13FF53FF93FFB3FFD3FFF3FFF3FB0
:10B6E000FF3F0000E0203420002020E02020202325
:10B6F00037202620210000800200040008001000EE
:10B700000002000400080400000200040008001009
:10B710000020004000800400000000800000004085
:10B7200000000020000000100000000800000004DD
:10B730000000000200000001000080000000400046
:10B7400000002000000010000000080000000400BD
:10B75000000002000000010000800000000801401D
:10B76000000C0140000C0140000C0140000C0140A5
:10B77000000C0140000C0140000C01400010014091
:10B780000010014000100140001001400010014075
:10B790000010014000100140001001400014014061
:10B7A00004080140040C0140040C0140040C014059
:10B7B000040C0140040C0140040C0140040C014045
:10B7C0000410014004100140041001400410014025
:10B7D0000410014004100140041001400410014015
:10B7E0000414014008080140080C0140080C014005
:10B7F000080C0140080C0140080C0140080C0140F5
:10B80000080C0140081001400810014008100140D8
:10B8100008100140081001400810014008100140C4
:10B8200008100140081401400C0801400C0C0140B4
:10B830000C0C01400C0C01400C0C01400C0C0140A4
:10B840000C0C01400C0C01400C1001400C1001408C
:10B850000C1001400C1001400C1001400C10014074
:10B860000C1001400C1001400C1401401008014064
:10B87000100C0140100C0140100C0140100C014054
:10B88000100C0140100C0140100C01401010014040
:10B890001010014010100140101001401010014024
:10B8A0001010014010100140101001401014014010
:10B8B0000000000000000000000000000000000088
:10B8C0000000000014080140140C0140140C014059
:10B8D000140C0140140C0140140C0140140C0140E4
:10B8E000140C0140141001401410014014100140C8
:10B8F00014100140141001401410014014100140B4
:10B900001410014014140140000000000000000069
:10B91000000000000000000000000000FFFFFF0F1B
:10B920000FFFFFFFFFF0FFFFFF0FFFFFFFFFF0FF25
:10B930000FFFFFFFFFF0FFFFFF0FFFFFFFF0FFFF15
:10B940000FFFFFFFFFF0FFFFFF0FFFFFFFFFF0FF05
:10B95000FFFF0FFFFFFFFFF0FFFFFF0FFFF0FFFFF5
:10B960000000004040000000000400000040000013
:10B97000000004004000000000040000004000003F
:10B98000000400004000000000040000004000002F
:10B99000000004000000400000000004000000401F
:10B9A000000400000000008080000000000800008B
:10B9B0000080000000000800800000000008000077
:10B9C0000080000000080000800000000008000067
:10B9D0000080000000000800000080000000000857
:10B9E000000000800008000000000020200000008F
:10B9F0000002000000200000000002002000000003
:10BA000000020000002000000002000020000000F2
:10BA100000020000002000000000020000002000E2
:10BA20000000000200000020000200000000006092
:10BA3000600000000006000000600000000006003A
:10BA4000600000000006000000600000000600002A
:10BA5000600000000006000000600000000006001A
:10BA6000000060000000000600000060000600000A
:10BA7000008002000400080010000002000400081A
:10BA800004000002000400080010002000400080B4
:10BA900004000000FF7FFFFFFDFFFFFFFBFFFFFF34
:10BAA000F7FFFFFFEFFFFFFFFFFDFFFFFFFBFFFFC4
:10BAB000FFF7FFFFFBFFFFFFFFFDFFFFFFFBFFFFA8
:10BAC000FFF7FFFFFFEFFFFFFFDFFFFFFFBFFFFFFE
:10BAD000FF7FFFFFFBFFFFFF401FFC02001E5A031A
:10BAE000C01CC403801B3C04401AC6040019630533
:10BAF000C01717068016E4064015CD070014D708B6
:10BB0000C012050A80115B0B4010DD0C000F900E77
:10BB1000C00D7510800C9012400BE014000A6517E0
:10BB2000C0081C1A8007FD1C4006002000051823D1
:10BB3000C003372680024E2940014C2C0000242FE0
:10BB4000C0FEC73180FD2E3400FB2D3880F81C3B31
:10BB500000F6003C8025151A40249A1B00231E1D68
:10BB6000C021B81E80205D20401F0C22001EC22371
:10BB7000C01C7E25801B3327401AFB280019B72ADA
:10BB8000C0176D2C8016192E4015B92F001447319F
:10BB9000C012C9328011353440108B35000FCA36BF
:10BBA000C00DF037800CFE38400BF439000AD23A51
:10BBB000C008983B8007473C4006E13C0005673DD4
:10BBC000C003DA3D80023E3E4001923E0000143F39
:10BBD000010203040500020304050001030405003B
:10BBE00001020500010203040405000102035505DA
:10BBF0000010AA1A55250030AA3A0000AA0A5515C5
:10BC00000020AA2A5535FF3FAA0A55150020AA2A66
:10BC10005535FF3F6465765F63616E31000000005B
:10BC2000018D0008B18E00082D8E00085D8C000883
:10BC3000258C00080000000014BC000820BC00088F
:10BC400064BC0008000000209C08000000070008F9
:10BC500094BD00089C0800203C150000588800088E
:10BC600038BC000801441359421B086D04211355C8
:10BC7000152A4006190801A713FB5C1408215D1B57
:10BC8000081B04012423286E420117020604050143
:10BC900003148020FF8BAA0A0201A415AA0A5515D5
:10BCA00000085920AA2A5535FF3F0735030105042E
:10BCB000060203127C1573FFFF04FF808001012D33
:10BCC000025F6402130A13598F52081201100C0507
:10BCD00004060203010103070505280B0102030402
:10BCE0000206070303040C3D0706040509191F1982
:10BCF0001904310506060B14AA1A02312E40FD392B
:10BD000069260211042F405F02041E405B2613D0F7
:10BD1000058A202ECD551555154039020187031689
:10BD2000D0071AFF01013B0261AA0C10080108A804
:10BD300034993F33137197391CA9100916E89122E1
:10BD40000312100A17401C12600A16901B011AA257
:10BD5000646B6D8F94012199D0019A5A14021AC80C
:10BD600002CBD007023A19164902892612C8DA0115
:10BD7000DA1AFF01C1227D130D0212103AFA0812DD
:10BD8000081CF401010812062BE8031012021B60C4
:04BD9000BC15B1002D
:020000040800F2
:10FC00004A46545A594D46312D4E3330202020203B
:10FC1000050406020301AA0AAA0AAA0AAA0AAA0A4B
:10FC2000AA0ADE3F00100000FF0131000301664612
:10FC300000400040513800400040004000400101B9
:10FC4000004000407A3B082708270827FF0033338D
:10FC50000201401F00016626B81E6626FFFFFFFF57
:10FC6000FFFF01010100010000000300000202008B
:04FC70000000AA5591
:04000005080000ED02
:00000001FF
